:1000000082E0128086401E1247ABA27F9251C27FCF
:100010007801127F06A251927FC251E53730E40485
:100020000F02F9D022E53720E4FA905903E0B50732
:100030000C905900E0B5061743370280B5D209127B
:1000400047AB128136E53720E0A85337FD80931E79
:10005000128288128C8D14FF12828880E58531838C
:1000600085328275F000438380E0F95301F6E5376D
:1000700030E405127E768001A305F0E054F66501B8
:100080007002DAEAE5F022905903E0B50702801722
:10009000853183853282438380E054F6F8127E7680
:1000A000E054F665006002D322C322128C8D14B591
:1000B000070280F31237CB853183853282438380F8
:1000C000E054F6F8A380D98531838532824383805A
:1000D000E053837F20E21B54F2FA207710E53030A2
:1000E000E30BE53820E20854F255027005C322BA4A
:1000F00000F5D322D2091237CB5337FE12828D126C
:10010000439C40061009EC02F9D0C209E53720E211
:1001100006303403433702EFB5F00D905901E0B5D6
:10012000060A43370102F9D00FA380D30E9059037A
:10013000E0FF12828880C5D2091237CB5337FE12F6
:10014000828D12829C400280BBC209433702C08369
:10015000C082905903E0D082D083B507099059003E
:10016000E0B5060880BC1F127E7680D61E128288FB
:10017000128C8D14FF12828880C55337FCE5303015
:100180000202800F225337FCE53030E3F7203403BE
:10019000207FF15337FE128204B4040122B403021B
:1001A0008004500DAE00AF0130340343370202F932
:1001B000D0B40509EEB5020280030E80E9904C42EE
:1001C000E0FE904C41E0FF128288306003EF03FFB5
:1001D00043370180D35337FC128204B4040122B4A4
:1001E00005028004400AAE02AF0343370202F9D091
:1001F000B40309EEB5000280031E80EC7E017F018E
:10020000B4370180E5905900E0F8905903E0F99087
:100210005901E0FA905904E0FBEEB5000050137C60
:1002200000EFB50100401B0CB50302801540130C14
:100230008010EEB50202800640047C0680E37C0359
:1002400080DFEC2212F38350038E3B221237CB8ED9
:100250003C8F3D905903E0FF12828812828D1282FA
:100260009C50098E3BAE3CAF3D028288EFB5F00A50
:10027000905901E0B506070E80E90FA380E00E90CB
:100280005903E0FF12828880D2D20902F9D0128C81
:100290008D15F085318385328243838022E0028090
:1002A000D3904CC4E0F5F0904CC3E0F5368043F9B0
:1002B000B420004006307121207850904C7CE01032
:1002C000E21DB90A0320F01130E10330710B904CAC
:1002D0004412712CE9F01283607536000273F5B98F
:1002E0000AE630F0F480E1E9B4210280C2B4401B98
:1002F00080BD12929F5014F9904C7CE020E2E8E916
:100300005021028006B402A72078A4904C78E065C2
:100310003670C6128D05904CC4E0F9128D05E06967
:1003200070B7128D05D536F13071AE790A904C77E1
:10033000E9F0904C81E0F5F080817403904C44F03A
:10034000028360740180F58DF090837E128C9A9008
:100350004C4810E70830E4085403904C49307115BC
:10036000F0904C48128375904C4AF0904C4912839F
:1003700075904C4BF022E0904C4412712CE0220F0F
:10038000000E016E826F837E117D127C13FF30712F
:100390001A904C2BE054FEF0780012FC0D02FC2069
:1003A000307108904C2BE0440180EC2274017918E4
:1003B00030711B207704904CD8F0904C447806E9BB
:1003C00083B4FF028001F009A3D8F4128360227481
:1003D0000280DB7403791E80D70121FFFF00010139
:1003E000FFFFFF00FFED5403904C4CF0D26D223024
:1003F0007147904C78E0FDA3B4012EE0CD12929F9E
:100400007430F9904C81E030E00AB921028025B9BE
:100410004020800BB902053078188018B9400530AB
:1004200072108010B9210D8009B40206E0F5F0A326
:1004300080C9790A904C77E9F022B8070F907FF4D1
:100440007401F075F0371273F5024196227F017E38
:100450000102F9D0D2D18002C2D1904C81A3E0C078
:1004600082C08390849730D1039084AEF5F0128CD3
:100470009AD083D082501330E00920D10330720A21
:1004800030710730E30C54F64233D534D0C2D10278
:10049000A49554F6523380F20004014804180588EC
:1004A0000728080B16B618E619761BD61CF5FF00B0
:1004B000F3010D02F3FF905F32E0B4400912C00077
:1004C00012897F0284C802000012FDE202475DD259
:1004D000D18002C2D1904C81A3E0C0D0C083C08241
:1004E00090851F2068039085C520E724304202D202
:1004F000E7F8E4930460191468204202C2E7600739
:10050000780512712C80EBA320D102A3A3127144B1
:10051000D082D083D0D0E5346003D534BBC2D122A1
:1005200081F885FF858273860686832A862E860457
:10053000638674860578869486869D86A18687A6BE
:1005400086A98608AE86BD868AC186D2868BEB8652
:10055000F2868DF98600878E07871587901C872E77
:100560008792358740879344875387995787688751
:10057000A66C877386AAA487A087ABBE87CD87ACFD
:10058000D187DB87ADDF87E987AEED87F787AFFBE4
:1005900087FF87B501880888BC0F881788BD1D882C
:1005A0002588BF2B882C88C02D883588C23B88427F
:1005B00088C349885488C458886E88C572887388EF
:1005C000C974888788FF818B888F880293889D886B
:1005D00084A788AE8886BB88BE888AC188C2888C7A
:1005E000C388D2888FD688DC8890E288E98891F029
:1005F00088F78894FE880D89FF780279FF02FBFF57
:10060000220079FD02FBFF20776A780612861D1012
:10061000710612FC2002C7A012FC2002898A904CAD
:100620002BE054F848F0780002FC0DD2798002C229
:100630007912F2A774503079027484904C41F0E53D
:100640002F781312FC0D12376612378612F3CC1274
:10065000EF7412BF4F1284C812A52C12E07612F26A
:10066000A702133C7810904C2CE020E50754C748B3
:10067000F012A50022780080ED904C2BE020E7F4EA
:10068000B2E7F012A5377B0112A5C312865D904B2D
:10069000D1E070FD22904C2BE030E7D880E2D26EA2
:1006A0008002C26E02475DD27D22C27DC26F227877
:1006B00020904C2EE054DF48F0780302FC0D7800C7
:1006C00080EF2077E9E530540C60E35330F343309A
:1006D00008800F2077D8E530540C60D25330F343B4
:1006E0003004E530781212FC0D02133220770343F8
:1006F0003040222077035330BF222077034330015C
:10070000802077035330FE2220770A7801904C3006
:10071000E054FE48F0222077FC780080F02077F546
:100720007880904C2FE0547F48F0780402FC0D2034
:1007300077E3780080EC7801904C32E054FE48F08A
:1007400022780080F37800904C32E054EF48F07843
:100750000702FC0D781080EF7800904C2DE054FDDE
:1007600048F0202E0302A47722780280ED309634E0
:1007700020773112878C780412861D12FC20128992
:100780008A1284C812DBCC12A4BA02F2A712F2A712
:1007900012EBEE74003031027403904C43F002EC23
:1007A0000510780E22904C2EE0540F60F72078F45C
:1007B000D278E52F781312FC0D12C7A00283EE78D1
:1007C00040904C33E0543F48F0780802FC0D78002C
:1007D00080EF7804904C33E054FB80EB780080F499
:1007E0007808904C33E054F780DD780080F478028C
:1007F000904C33E054FD80CF780080F4788080C145
:1008000001CC207703433002222077035330FD22AE
:1008100020770AD27A02DCC4207702C27A222077BB
:10082000FCD27B02DCC4207702C27B22222220770A
:10083000ECD27C02DCC4207702C27C22780179FFF2
:1008400002FBFF780079FE02FBFF7820904C2FE03E
:1008500054DF028727780080F37810904C2EE05404
:10086000EF48F0780312FC0D30780312C7A022780D
:100870000080E82222781012FC62904C0350039012
:100880004C07E054EF48F022780080EB4330102210
:100890005330EF227402303102742042392274FD49
:1008A00030310274DF523922D26C12A7038005C2A4
:1008B0006C12A6B6E53030E3BB021332D27F22C2FF
:1008C0007F2222227800904C34E054DF48F07809EF
:1008D00002FC0D782080EF207702D27E2220770262
:1008E000C27E222077034330802220770353307F5B
:1008F00022207703433020222077035330DF2278F1
:1009000078904C2DE054FE48F0780202FC0D7800FF
:1009100080EFE4202E13304104740B800C12FE7E15
:10092000904C025003904C06E0540FF5F090893E35
:10093000128C9A400274642013FDF51AD21322001F
:10094000280132023C03460450055AFFB83D0578A1
:100950000502896FB83E028003B83F207800E53475
:1009600014600C904C83E0B4030050101460010834
:1009700012861D12FC201283EE02898A223071FC3D
:10098000D2781287A012EF001287A012A56E12EF84
:10099000001286A912875712C00D12AE0212C1AC06
:1009A000D27E1272FB12458C1245BC12EFE7127315
:1009B00099D27F905C81303103905CD6E05408F886
:1009C000904C2BE054F748F0780012FC0D1286D2C0
:1009D00012871C12870712888B1288F01288011266
:1009E00086F20288E2C27512F315809F78050286AE
:1009F0000B7804904C32E054F302874C780880F373
:100A0000340080EF22C26F10600122AD06904C418D
:100A1000E003F87484C398FA1237CB128C2579005E
:100A2000128A25028A48AD06128B26543F49CCE033
:100A3000CCF06C54C0227940207705E53720E6F5EC
:100A4000128A25C26F60EED2601247F87B0502A4BD
:100A5000F9798080E379C080DFE86003B801112074
:100A60006808700C20770602AA4BB8013F02AA342E
:100A7000B804112068028007A23192D512AEA47882
:100A8000000289F2B8051D904C32E020E315306871
:100A90000BA23192D512AEA3780480E530230478FE
:100AA0000880DE22B8020A3068077401904C71F0A9
:100AB000223068EFB80803C24722B80903D24722A0
:100AC000904C0AE0B8121120310720E1D6D2E08024
:100AD0000520E0CFD2E1F022B8130F20310520E14C
:100AE000C2800320E0BD54FCF022B80A08E8906000
:100AF00048F002AA71B80BAB20770302AA0E02AA33
:100B0000C0EDB501005006B50000400122D322A37C
:100B1000A3E493B4FF0122C398A370F393FAA3E470
:100B200093F5838A82E473C000C002C0068D06D2AA
:100B3000D512F9D7A3E0D006D002D00022C006AE6D
:100B40000512FB5ED00620502FC252128C48307026
:100B500053306925E53030E320438380E053837FC1
:100B6000C0021280D3D002400CE4F0438380E054F2
:100B7000F7F053837FA3DAE1223069028003207FFC
:100B800023438380E053837F20E215E4F043838096
:100B9000E054F72069025401F053837FA3DADA228C
:100BA000D25280F8307010E4F0438380E05401F0BA
:100BB00053837FA3DAF122E4F0438380F053837FF1
:100BC000A3DAF522128C48207F05E53020E312E9F4
:100BD000F0438380E054014540F053837FA3DAE77C
:100BE00022438380E053837FC0021280D3D002402F
:100BF000EC80DC128C48438380E049F0A3DAF722D2
:100C000030052050048E058005905901E0FDA902B1
:100C1000128B2654C06003E903F9128C48D00543B7
:100C20008380AC83AB82128C48E4F0305110B90061
:100C300002800B19128D06E054F7A3128D06438330
:100C400080F053837FA3DAE122C000C002C006AE69
:100C500005D2D512F9D7F5838A82D006D002D0000A
:100C6000E802712CE4F0438380E53030E305E05482
:100C7000F78001E4F053837F205003A38003127EAA
:100C800076DCE122904C82E0F80582E0F922904C7B
:100C900041E0043060020403F5F022E493A3B4FFC2
:100CA0000122B5F004E493D322A380EFF8C4540FDB
:100CB0006008C3C89406C8D5E0F922904CC3E06030
:100CC00043F9A3E0FCA3E0FBB90330A3E0FAEC9402
:100CD00030C4CB94304B78FFB426005028128CAB34
:100CE000E8C0F075F00AA4D0F0CA24D02A501578D4
:100CF000FF22C4F8EAC394304880B1EBFAECC39405
:100D000030B901EEF822A3C582CBC582C583CCC51C
:100D10008322307035E87031800320722C904C2C87
:100D2000E05407B407043096010423FC908DC2936D
:100D3000CC0493FBAA0390EC0130310390EE01EC5C
:100D400083F0A30CDBF9128F12227B037C0F80E46B
:100D50001B2F5A1B5B3F313B32631B5B3F313B30E8
:100D6000631B5B3F36631B5B3F31323B373B313BA1
:100D7000313032631B5B3F37639B3F36323B313B45
:100D80003B3B363B373B383B39639B3F36323B314D
:100D90003B323B333B343B363B373B383B39639B41
:100DA0003F36333B313B323B333B343B363B373BC7
:100DB000383B393B31333B31353B31363B31383BC6
:100DC000313963120719072005250E3305381149FB
:100DD000155E265E247B0C7C0A3096077C0A2097E1
:100DE000027C1690EC0130310390EE01EC83F0A30D
:100DF0000CDBF97A0C028F129B3E31383B31313BD0
:100E0000E03B30639B3E31393B31313B303B30631B
:100E100090EC0130310390EE017A00749BF0A30A4C
:100E20002220680D908E27028B0E06A88E05658FF6
:100E3000FFB80F5412AE027B0D30232992D1A2319C
:100E400092D512AE6740097B132072197B0D801575
:100E500012AE7840097B1220720B7B0B80077B0A55
:100E600020D1027B0B128E0F786E743FF00AA3EB39
:100E7000B40A00400B75F00A842430F00AA3E5F0B0
:100E80002430F00A028F0E22B819063071F9028F51
:100E900075B81A03028F85B80603028EA8B8370307
:100EA000029004B838E102902F7852128E0F306809
:100EB00005743FF0A30AEE306E11C082C0839059D2
:100EC00000E014FBC3EE9BD083D082307702740124
:100ED000128F2E743BA3F00AA3EF306E11C082C0B4
:100EE00083905903E014FBC3EF9BD083D082128F11
:100EF0002E30681B743BA3F00AC082C083904C4321
:100F00009B0430310224FDD083D082A3128F2EE8BF
:100F1000A3F00AEA30310C90EE00F0905FC1E0D20D
:100F2000E2F02290EC00F0905FC0E0D2E2F02253B9
:100F3000D03FFD540FD4CDC4540F6014FBED2416E4
:100F4000D45002D2D1DBF7CD30D1050A7431F0A3F1
:100F5000EDC4540F10D10260052430F00AA3ED5403
:100F60000F2430F00A22128E0FE51F600274031264
:100F70008F5E786E80997B14904C2FE020E6028083
:100F8000027B15028E6420710122904C2EE0540FDA
:100F9000FA90EC0130310390EE017C607B05EC832C
:100FA000F0A30CDBF9EA7A0904FBB40A00400874E8
:100FB00031F0A30AEB24F62430F0A32072041A1AAD
:100FC0008038743BF0A3C082C0832018FD78A079DC
:100FD0000F904BE67401F0904F08E0F5F0E0B5F0AB
:100FE00008D8FAD9F87433800B12F3BF5004743068
:100FF00080027438D083D082F0A3746EF0028F1216
:10100000F83F32373B128E0F743FF0A30A7435F06D
:10101000A30AC082C08312906470047433800F747A
:1010200030202605303107800320310274388026B5
:10103000128E0F7C287B04EC83F0A30A0CDBF8C033
:1010400082C08312906470047430800A90670CE050
:101050007B3160010BEBD083D082F00A786E028F77
:101060000E3F35373B907FF5E4F0907FF174FFF051
:1010700012A64012F2A7907FF1E00460FC90670B8B
:10108000E02202913F206BFA3071F775F084904CAA
:1010900082E0B4020050EBA3E0B4600050E404F03E
:1010A000904C84E0B4030050D9A3A3E0B4030050F3
:1010B000D1600114F0904C7FF0780A6002780690BD
:1010C0004C85E0B50009904C87E0B402B580115022
:1010D0006FB40102806A7001E8B405005002C2F2E8
:1010E000904C87E0B40300505730F20BA3E070023D
:1010F0007414B415005049904C89E0B4020050407B
:10110000F0904C81E0B500028006904C847402F0AF
:10111000E87012904C83E0B40106D2F574028009A5
:10112000B46002801B904C83E0904C76F0904C8130
:10113000E8F0E5F0904C93F07534001293288002AB
:10114000D26B740402743D306B0302962D904C9365
:10115000E0F5F030F7030291F220F405D2F4129199
:10116000C3D2F6BD3B0853F0F4129337805320F3FB
:1011700050BD2F23C2F020F117904C95E004F020D1
:10118000F207B4010DD2F18009B40306D2F1800256
:10119000D2F3129356802A20F027BD3F004022BD93
:1011A0007F00501DED24C1FDE534B40A0730F10B7A
:1011B000D2F3800D12936005348006D2F08002D203
:1011C0006B02962D904C84E0FB6003B4020BC0F0E0
:1011D000C00512A578D005D0F022904CC3E004FAE7
:1011E0007B787C4CE0FD128D05E06D7005128D055D
:1011F000DAF222904CC312926110D54B10D10489BF
:10120000528041502EFA904C81E030E00EEAB42139
:10121000028017B4400C307209800FEAB402052036
:101220007808800FB440033072F8904C77F0129237
:101230004B800912924B904C77740AF0E9547FF579
:10124000F075360002962DC2D10291BE7A04904C00
:1012500078128D06904CC3E0128D05F0128D05DAE0
:10126000F622C2D1C2D5A9F0BD3000500F0536E537
:1012700036B40300507B12712CEDF022D2D105362A
:10128000E536F012712CEDF0C0051291D9D005EAC7
:101290006006904C847402F0904CC4E0F5F0E536A2
:1012A000B4012F904C2EE0540FF5F09092F3E4939C
:1012B000A3B4FF01226D70149310E708B42103203A
:1012C000780AD32265F07004740280F6A380DF22CE
:1012D000C322B402FBE5F0B425F6BD35047420D377
:1012E00022BD36EC904C2EE0540FB40FE374028014
:1012F000EED2D522420130033C4041213E224181C1
:101300007482518345843684438535854B86348782
:1013100059883D893D8A488B378B458C368C608C4B
:10132000528D5A8E39836084FF7A28904C9AE4F06B
:10133000A3DAFB904C95F02230F612904C76E0B494
:10134000610CD26B12A69712F2A70213322210F58B
:101350000312940E129328904C7574FEF0753400AD
:1013600022904C75E0F923F0E534B40800504E7833
:10137000007B80AC34904CB130F203904CBD20F136
:101380000F904C95E023FA232A23904C9912712C4C
:10139000A3088836E059FAEB23FB5D03D536FCAC95
:1013A000340C23DCFD4AF0A320F207A3F0A374045D
:1013B0008002740220F1027406B500D42278007B0A
:1013C00080E53424F8FC904CB230F203904CBE20FF
:1013D000F110904C95E023FA232A23904C99127136
:1013E0002CA3A3088836E059FAEB23FB5D03D5361E
:1013F000FCAC340C23DCFD4AF0A320F207A3F0A3DD
:1014000020048002740220F1027406B500D42290F8
:101410004C76E004F0904C9414F012A57312F2A7ED
:10142000904C94E070FD2212942E129465806B20F3
:101430006B33307126904C2FE020E61F75F0009042
:101440004C82E0B40104D2F08002500FE534B401C4
:1014500002800BA3E0B40101224003D26B22904C26
:101460002FE0D2E6F022206B3020F020801F904C3D
:10147000C3E0C0E012ECADD0E012712BE53630F1E4
:1014800006700474FFF534F0A3E534F02212ECADDD
:1014900075361EE4F0A3D536FB22206B06E5F090EE
:1014A0004C93F0740502743D7911E8B41100401DAD
:1014B000B416028018404009B41B0280104038095D
:1014C000B41E028008403009B42300402AD2F7023B
:1014D00096297930EDB4300040F5B43A00401879DF
:1014E00037B4410040E9B44700400C7957B461007B
:1014F00040DDB4670050D8C399221294D120F54D35
:10150000EBF20AC4FA129523EAF002951FFA12953B
:1015100023E04AF00536E5362534D2F17002D2F5E3
:10152000B2F28026A23112ECA4E536253412712CD9
:10153000227830793A128B004010904CC3E004B40A
:101540000300500EF012712CEDF002962D30F102D6
:10155000C2F5D2F780F4206B0C904C93E0F5F0BD0F
:101560003B0612959A02962D20F7FA20F68CBD2F95
:10157000C0029573904CC3E0128CBA1294A7904CA1
:10158000C3F0D2F6C0E012ECADD0E012712BE4F063
:101590001295DC8D3475360002962D20F70630F654
:1015A0000312946D904CC3E4F053F0307536002272
:1015B000AB05AA00A23112ECA4EC12712CE0F9A246
:1015C0003112ECA4EB12712CE9F00C0BD8E612EC02
:1015D000ADE534230412712CEDF02AFD22C2F57D15
:1015E000007CFF7534007A0012ECADEA12712BE03A
:1015F000F9A3E0FBB9FF06BBFF03D2F522E9601BAC
:101600007CB504005015B5050AED295003D2F5222A
:10161000FD80CE40068A34AC03A8010ABA0FC97413
:10162000FF6C60051295AF80B82215811581904C32
:1016300093C5F0F022C2D1904C2EE0540F90966EDC
:1016400023FA93CA0493F5838A8220D101A3E493F9
:10165000B4FF02D322B5051330D106A3E493FDC332
:1016600022E582158270F5158380F1A3A380DF8EB9
:101670009690969496A896BE96CC96E096F296068C
:10168000971C971C973697BE9694964C975E97FF3B
:10169000FFA323FFFFA323E040B05BE75CA75DE966
:1016A0007BF97CE87DA87EFFFFE040E25BE75CEA37
:1016B0005DEE5EF460E97BF97CE87DFB7EFFFFC6B2
:1016C0005BD85CC55DE67BF87CE57DFFFFC45BD63F
:1016D0005CC55DDC5EE960E47BF67CE57DFC7EFF5D
:1016E000FFA740C45BD65CDC5DE47BF67CFC7DDF61
:1016F0007EFFFFA323BE40835BBD5C7C5DA87B8433
:1017000071BC7DB47EFFFFA323A740B05BE75CE91B
:101710005DF960E07BF27CE87DEC7EFFFFF923E081
:1017200040E95BE75CEA5DEE5EE85FF460E47BF66F
:101730007CFC7DFB7EFFFFC940C45BD65CC55DDCE5
:101740005EE960E47BF67CE57DFC7EFFFFA323A7DA
:1017500040A15BD15CBF5DB07BF17CE77DFFFFC347
:101760005BC75CD55DE37BE77CF57DFFFF906B2974
:10177000128C9A5006301003029928906ACE128C6F
:101780009A500DD2D5B8BF00500302992B0298157C
:10179000791B906B0112710F600122909D46201001
:1017A0000E201C08E57F30E206300203909E86ABD7
:1017B0007E530B0F0BE412712CE493F9543FDBF6CC
:1017C000A3C082C083906B42C954C0232375F01B11
:1017D000A412712CEA93FBD083D082C00AB9010213
:1017E00080170A79007C037808E49333500109DA02
:1017F000028006D8F6A31C80EED00AEB5018EC123B
:10180000992CA3E4937003A393A3D9F6C57EA2E415
:10181000C57E5002E493C0E0904D3E302603904ECA
:101820003EE020E005D0E0025F64D0E07B01F5F00F
:10183000201018201C0B30020FC57FA2E2C57F507C
:101840000DB43C39743E80350298E00298E2C57EC2
:10185000A2E4C57E5027C00AAA7E530A0FBA04111B
:10186000B47D028008B47B028003B47C0ED00A8071
:1018700070BA050280EABA0C0280E5D00ABA1000FC
:101880004058BA1400AA7E530A0F5044BA0307B452
:101890005C4874FF804BBA0405909FFF802FBA0507
:1018A0000590A0048027BA060590A009801FBA0BF6
:1018B0000590A00D8017BA0C0590A012800FBA0EEB
:1018C00007B47C16745C8019BA0F0F80F4029FEC89
:1018D000BA0307B47B0474FF800712711B504D24B8
:1018E000E080491299BC400F906B1C128C9A4039D1
:1018F000E5F012711B400BB2D530D5030297AB0255
:10190000E5B9202E2220481FF812FE8CE8400FB4C3
:101910007304D2038005B47105C203026508B46D77
:10192000067B00747E800224A00299ACFCB4800087
:101930004012202E03304803304D7B906F0C128CE8
:101940009A403DECB47F2C3001221260C4806812B2
:101950006157500302603A904D2F302603904E2F6E
:10196000E0A2E5747F504A7408FC8045202E0330C5
:1019700048DD1B30013BB409028032B40D08802DD4
:10198000302803FCD225203305B4FF08802C1267D1
:101990008AD22522904F4230280AD2251299E0405F
:1019A0000C0260BBF0D228D201D21B800A1260C4A4
:1019B000FC20E706C2D1221270FAD2D12290966E94
:1019C000E57E540F23F893C80493F5838882A3E43B
:1019D00093B4FF03E5F022B5F004D3E5F022A38031
:1019E000EDC57EA2E4C57E5009F5F0E0F9909D17A3
:1019F000803EEC129A5CF5F0E0129A5CF9909A65E0
:101A0000227E540F142312712CE493FAA3E493F56D
:101A100083EAF582E4936018696007740312712CFD
:101A200080F2A3E49365F06004A3A380E7A3802A77
:101A3000A3E5F0C3995004E9C5F0F9E4937003C33A
:101A4000801A696007740312712C80EFA3E4936518
:101A5000F06004A3A380E4A3800093D322B4B00277
:101A6000742AB4810022839A749BBB9AE49A459BA2
:101A7000BE9B139BFC9BBF9CBF9C969CE49A749B53
:101A8000499CEB9C002022222D4C232D6C233D4CA5
:101A9000233D6C2320272741414061614041614043
:101AA00028285B2F3C5C29295D205E5E2060602831
:101AB0002D7B2F5E7C292D7D207E7E000020222222
:101AC0002B2B232027276061405E615B2C635C5ECB
:101AD000655D5E695E5E6F6027657B60757C6065D5
:101AE0007D5E757E0041455B61657B0041414061E3
:101AF0006140416140205E5E206060207E7E202249
:101B0000222B2B232027272F4F5C2A415D2F6F7C10
:101B10002A617D00333440696A5B31325C662D7C1A
:101B200031347D002022222D4C232D6C233D4C236B
:101B30003D6C232F5E5D206060202727205E5E22A3
:101B40005E7B27277E00002022222B2B23202727A5
:101B500061614041414041614022415B224F5C2A2A
:101B6000415D22555E27656022617B226F7C2A6180
:101B70007D22757E00002022222D4C232D6C233DDA
:101B80004C233D6C23202727606140305E5B205B47
:101B90005B202A5B2C635C21735D21535D6F735D59
:101BA000536F5D4F735D4F535D30735D30535D20F8
:101BB000606027657B60757C60657D205E5E0000EF
:101BC0002022222B2B232027272153402173406FD3
:101BD0007340536F404F73404F5340305340307306
:101BE0004022415B224F5C22555D205E5E2060609A
:101BF00022617B226F7C22757D73737E0000202220
:101C0000432D4C232D6C233D4C233D6C2320272753
:101C10002173402153406F7340536F404F73404FC7
:101C20005340307340305340305E5B202A5B205B72
:101C30005B2C635C27655D205E5E75866061867BDC
:101C40006F867C65867D69867E00002022222D4C71
:101C5000232D6C233D4C233D6C23202727217340EB
:101C60002153406F7340536F404F53404F73403088
:101C7000734030534021215B4E7E5C3F3F5D205ED0
:101C80005E206060305E7B207B7B202A7B6E7E7CCA
:101C90002C637D207E7E00002022222B2B232027F8
:101CA0002727454022415B224F5C2A415D22555E39
:101CB00027656022617B226F7C2A617D22757E0010
:101CC0000020222260752320272760614027655B62
:101CD0002C635C5E655D5E695E60655F5E6F602261
:101CE000617B226F7C22757D5E757E000020222242
:101CF000202727616140416140414140417E5B2C8A
:101D0000185C4F7E5D205E5E206060617E7B2C6390
:101D10007C6F7E7D207E7E00002022222B2B2320C4
:101D2000272761614041614041414028285B2F3CA9
:101D30005C29295D205E5E206060282D7B2F5E7C03
:101D4000292D7D207E7E0001019CA360A4006000FF
:101D50007BFF005D5B007D5D005CFF0040FF5E007F
:101D60007C5C00FF23158000E42000FF7E005C5DAA
:101D70002300806000FF5C007BFF0E8018F4207E53
:101D80002B277D227C7B272D148018F42000FF7EDA
:101D90002B00FF5E7D007EFF7B7C272D1A8019F6CD
:101DA0002000FF7E007EFFFF7A007D402B007B5DE0
:101DB000007CFF23792D0E0000C40000FF5B00FFB4
:101DC0005D00FF5CA4E1E4AC2000866000234000DD
:101DD0005D23007DFF5E005C5B007B5D71007EFF2C
:101DE0000060FF612A007CFF188019F6202127007F
:101DF000825E7A005FFFFF0040FF005BFF24792DC9
:101E00005B8019F620212700825E7A007DFFFF00AB
:101E10007BFF007CFF24792D1A8018F42000FF7EC0
:101E20002B00FF5E007D5D007E23007BFF007CFFBA
:101E3000272D0E8018F4207E2B277D227B7C272DDA
:101E40009CA360A40060007BFF005D5B007D5D00E3
:101E50005CFF0040FF5E007C5C00FF23168018F4EE
:101E600020005D402700FF5D602BFF007CFF007DB0
:101E7000FF2D158000F40000FF5C2700FF5D00834C
:101E80007E007CFF00FF5B4C00F000E02A28295F09
:101E90002C2E3F4C00F000E02A28295F2C2E3FD149
:101EA0008010840000FF7E005BFF007EFF00FF408B
:101EB0005CB2F0E4E0FF222F3F2A28295F00FF5B9D
:101EC00000FF4000825E00FF7C272EFF4FA308F436
:101ED000004022262F605D5E5C5B2A53A308F4005D
:101EE0004022262F00FF605D005EFF5B5C2A58B336
:101EF00009F6005E220040FF262F605A005D5C2A32
:101F000060005CFF27595EB0F0C4E000FF7E00FF78
:101F10004000FF232A28295F00FF7B00FF7D005D32
:101F20007C2C2E3FD4801CCC2000FF7E005BFF2B3E
:101F3000513D264100405C2165FB09F620FF2B2224
:101F40002A005C40262F0080605A007D5C00FF7EE6
:101F5000007B5D007C5B00FF235900FF5F63FB0992
:101F6000F620FF2B222A005C40262F0080605A00BA
:101F70005F5C00FF7E00405D5B00FF235900FF5F58
:101F80005CB308F400FF2200FF40262F00FF600032
:101F90005D5B005E5C005BFF005CFF2A4FA308F402
:101FA000004022262F605D5E5B5C2AD18010840099
:101FB00000FF7E005BFF007EFF00FF4058B308F487
:101FC00000005B5C2200FF23262F00FF5B5E2AFFE0
:101FD000005CFF7E5982F0F42000FF7C222A282931
:101FE0005F6000FF7D5E005CFF00FF7B3FE493B419
:101FF000FF05E5F00298D9A3B5F0F224E002992B91
:10200000007B7C7DFF7E7B7C7DFF7D7C7BFF7D7EFE
:102010007C7BFF7B7C7DFFC082C083758CF8758ADA
:10202000C4E581B478004027B47E005006202B1F01
:1020300020581C75D0007581477423123B6474814D
:10204000123B6474A7123B64740A123B5780E4E5A8
:102050001720E20720E60B7411800920E60A7410AD
:10206000800274012517F517103005D23002A1EC5B
:102070000000000000000000000000000000000060
:102080000000000000000000000000000000000050
:102090000000000000000000000000000000000040
:1020A0000000000000000000000000000000000030
:1020B0000000000000000000000000000000000020
:1020C0000000000000000000000000000000000010
:1020D0000000000000000000000000000000000000
:1020E00000000000000000000000000000000000F0
:1020F00000000000000000000000000000000000E0
:102100001B000000000000000000000000000000B4
:1021100000000000000000000000000000000000BF
:1021200000000000000000000000000000000000AF
:10213000000000000000000000000000000000009F
:10214000000000000000000000000000000000008F
:10215000000000000000000000000000000000007F
:10216000000000000000000000000000000000006F
:1021700012A2E8E545540FB40809201D085345F0A4
:1021800002565D0545D083D082D0D0D0E032E5162E
:10219000904BE82582F582E0D51602C21802A2848F
:1021A00074E302A284904BE974A7F0E51330E422B3
:1021B0005313EF904D2D302603904E2DE030E60462
:1021C000748680027482904BEAF0751602742302C2
:1021D000A2821513904D2F302603904E2FE030E051
:1021E000E380DD74E102A284749902A284201D348C
:1021F00030993120189820196F20137C101A46103E
:1022000018E110142210159D1017DD101692904B36
:10221000E6E06010E4F0904BE97480F0751601740C
:102220000A02A28202A16F904BE9E520540F44807C
:10223000F0904BEB640FF0904BEA7413F0751603BB
:10224000741102A282E513541F70B4904BE9749983
:10225000F0A3749FF07486305C027482904BEBF0B4
:10226000751603741B02A282741F2516830516704F
:1022700014C2197516008011E51A83051A7006C27A
:10228000138006D218C299F59902A16F0A801281B3
:102290001A8022803A8142814A825A8262826A820C
:1022A0007282007864867A64867C64860078648AA8
:1022B0007A64867C64860078648D7A64867C648621
:1022C0000078649E7A648A7C64860078649E7A646E
:1022D000947C648C0078649E7A649E7C6498007818
:1022E000649E7A649E7C649E0010980122201E11D8
:1022F000904F08E00454074400F0F582E599F0059A
:10230000A022202F1A907F00E06013F90582E0F5EB
:102310008212A35AE582907F01F01582C9F022E46F
:102320002275A07E787EE2FB08E220750D20730AFC
:10233000C39B5002247EB4011222A803CBC39BABE3
:10234000005002247EB40400400322A803EDF2EB07
:1023500004B47E03D37400787EF22220752B2073A0
:102360002875A07E787EE2FB08E2C39B5002247EA3
:1023700014B501004013EBF8E0F2E804B47E0274F7
:1023800000787EF20582D9EF22E0FD12A3205004EE
:102390000582D9C722202F09907F017402F0302FC7
:1023A0002BC003C00075A07F7870E2FB08E2C39BDE
:1023B0005002241EB4010280ECA803EDF2EB04B439
:1023C000700274527870F2D000D00322907F00E047
:1023D00004F0042582F582EDF02212A6B3202F1816
:1023E000907F017402F01582E02402F02582F582CC
:1023F00074FFF00582ECF0227DFF12A3A0ECFD80BB
:10240000DD12A320400312A394227C0002A4107CBE
:102410000112A3DC907FF3E070FD74FFF012A301C2
:1024200070FB227C0280B67C0312A6CB202F1C906E
:102430007F00E02403F0142582F582EEF00582EFA0
:10244000F00582E53554C0F002DCC4AD0612A3A04D
:10245000AD0712A3A0E53554C0FD12A3A002DCC451
:102460007C04C26412A3DCAD03BBFF0302A4AB0275
:10247000A39D7C05D26480EC7C067B00904C2DE013
:1024800030E1010B02A4997C077B00904C2DE030D9
:10249000E2010B02A4997C08AB3312A3DC8B05028A
:1024A000A39D7C0902A4107C0A02A4107C0B02A349
:1024B000DC7C0C02A3D97C0D02A57A7C0E02A3D988
:1024C0007C0F02A3D97C10E53523235403FB02A51E
:1024D0007A7C1102A3D902A59F2077FA7C1212A35D
:1024E000D9BB03004009907FF3E070FD74FFF0ADAD
:1024F0000312A39D12A30170FB222077D97C1380C5
:10250000017C14904C2CE023C4540790A51293FB3B
:1025100002A57A00010204007C1512A3D99059008B
:10252000E0FD12A39D905901E0FD02A39D7C167B66
:10253000003079010B02A57A7C177B00904C2BE0D0
:1025400030E7010B02A57A7C18ABF002A57A7C1962
:1025500012A3D9880512A39D128C83890502A39D1D
:10256000227C1B12A3D9907CA0E004F002A3017C82
:102570001C02A3D97C1D02A3D97C1E12A3D98B05F2
:1025800002A39D7C1F80F47C2080F07C2112A3D9C3
:10259000905903E0FD12A39D905904E0FD02A39D14
:1025A0007C2202A4DD7C2380D27C2480CE7C25800A
:1025B000CA7C2612A3D902A4137C27BB01BD12A595
:1025C0007A02A4137C2880F37C297B00904C2DE0B8
:1025D00030E3010B02A4997C2A02A3D97C2B12A51B
:1025E0007A02F2A73077047B0580B57C2C12A3D940
:1025F000AD0212A39DAD0012A39DAD0312A39DAD2C
:10260000F012A39DAD3B12A39D02A4137C2D02A446
:10261000997C2E12A3D9AD0312A39DAD0212A39DE6
:1026200002F2A77C2F12A3D9AD0302A39D7C300236
:10263000A3D97C3112A3DC02A4137C32AB1F02A409
:10264000997C3302A3D97C34800E7C35800A7C3699
:1026500080067C3780027C3812A3D902F2A77C392D
:1026600012A57A02F2A77C3A7B003077010B02A513
:102670007A7C3B02A3D97C3C02A3D97C3D02A3D93E
:102680007C3E02A3D97C3F02A3D97C4002A3D97C23
:102690004102A3D97C4280C07C4312A3D902A41377
:1026A000306C10904CD6EFF0904CD7E07005740170
:1026B000F0800422306C14202F1112F28D70FB90E8
:1026C0007FF77401F0907FF7E070FD22306C32905C
:1026D0004CD5E0CEF0CEB50616E53730E417904C79
:1026E000D6E0CFF0CFB507028017401502A3D9126C
:1026F000FE3702A3D9904CD7E07006907FF87401A2
:10270000E002A3DC904CD5EEF012FE37904CD6EFF1
:10271000F022202E0CC25712A71BD25712A7DD4061
:102720000122B4FB0512B18B802E4066B4FD07A2D6
:10273000571278808022B4FF2720570D433A0412A5
:1027400055CC905FC04013800B433A101255D79080
:102750005FC14006E0D2E0F08027E020E023806205
:10276000B4FE27907CA0E0FB541FB41B16EB04F0D2
:10277000907CCDE52AF0205705533AFB8003533A6D
:10278000EF8055A25792D502AA30B4FC052057EE2F
:1027900080E712A8084041E53AA2E2305702A2E4DD
:1027A0004021302333907CCDE0652A20E71412AD20
:1027B000FF500F907CD074D1F012A7DD12AF8212BF
:1027C000A7F62220411212A7DD7B01205705125CDB
:1027D000EE8003125E0F50EA12A7F602A71B907E4E
:1027E000FE305703907DFEE0F5F00582E0B5F00184
:1027F00022D3F582E0FB22907EFF305703907DFFCD
:102800007804B4FE027480F022907CCCE02057055E
:1028100010E007800E10E1028009F012A7DD24FA13
:10282000F0801612A7DDB4FA10907CCCE02057059A
:10283000D2E0F0D322D2E180F9C322E514604D90BA
:102840004C0AE020E12B20E00F907CA0E030E60570
:1028500020E71E80032026191255CC402F1253DF8B
:10286000125CE950071254FDE51470F1905FC080CE
:10287000171255D740161253DF125E0A5007125432
:10288000FDE51470F1905FC1E0D2E0F022907C9EF3
:10289000E030E505C2D512AE8D907C9FE030E505B5
:1028A000D2D512AE8D12ADFF400122907CD074D1F2
:1028B000F0907CA0E0F8547F700A12AA96400512AE
:1028C000AA9D50E6E8A2E730E609303101B340DACC
:1028D00002A9E530E511541F700D400512AA96803B
:1028E0000312AA9D40012212AD03907CCFE060F656
:1028F000D22102F818A23192D512AE64500B12AE5A
:102900007C500512ADFF40092212A30170FA024E5D
:10291000FD7440907C9E303101A3F0A23192E7908B
:102920007CA0F0907CC7E0600302A98D907CCFE092
:102930006005D22102F81874D1907CD0F01255862F
:1029400050C61253761253FE12B98840EAED20E7C2
:102950000AB41B1112AF8274018025B4A000400A92
:10296000202202C2E712AF8280C220780320221602
:10297000741B12AF82ED64C012AF82B45BAE7402FE
:10298000907CC7F080A3B49BDC12AF8280F012551C
:1029900086507B12537620E766B41B028061125387
:1029A000FE12B98840E8ED12AF82907CC7E0FB04CC
:1029B000F020700EBB0148EDB45702803DB4583F83
:1029C0008024EDDB06EDB45B3680C3DB10907CC861
:1029D000B43404E4F080B7B43525F080B1B4691F95
:1029E000907CC8E07014904C32E0C2E3F0904D321D
:1029F000303103904E32F012B1B8907CCFE4F090B9
:102A0000EEC7E4F0904C32E030E30302A92B2278C9
:102A100008A23192D512AE645016907C9E30D5013A
:102A2000A3C3E058700A75A800E048F075A887D3E2
:102A300022781080E5EE904C6DF0A3A3E4A277928B
:102A4000E7A25A92E6F0C25A780280C5780480C1A3
:102A5000126A765015A226904D2B5003904E2BE013
:102A600020E5077401500104800B780480ACA22695
:102A70008002A231E4907CCEF092D5C33023B1E441
:102A800030D50104907C9DF074019060B8F078011D
:102A900012AA19B2D58083907C9EC2D58005907C05
:102AA0009FD2D5E0601B75A800E020E516D2E710A4
:102AB000E06B10E23010E13D10E31610E40A75A857
:102AC00087C32212AE8D80DBF075A8877B1B02AB1B
:102AD000B6F075A88712ABB4793FE3F0E430D502C5
:102AE0007403A3F022F075A88712ABB47401F079D7
:102AF00043E3A3F022F075A8877B0112ABB612AABC
:102B0000127401A3F0796DE3A3F0E4F309A3E3F0F9
:102B100009E3A3F0E4F309E3A3F0E4F322F0638212
:102B200001E06481F075A887E8907CCBF012EBEEB1
:102B3000E4907CC2F012ACE2907C9DE0A2E092D5E1
:102B400012ACCC904C00E0C44402540EFA30960A09
:102B50007933E330E0047B1A8065E4906048F0EA62
:102B600030E2067B1412ABBE2230E3047B0D80F50D
:102B70007B0612ABBE7401F0907CBCE0B403004055
:102B800007904C01E030E2077900907CBC80057929
:102B900024907CBDE0907CB6F0907CBE75A0617AFC
:102BA0000412F3B8907CBE12ABAAA3E0FAA3E0C370
:102BB0009A04F0D3227B0612EBEE12ACCC7A0079A9
:102BC00032E3F5F003C454604BA2D592E7907CA0A9
:102BD000F0F8A3E5F054F14AF5F0F0793EE3A2E015
:102BE00092D1792BE3A2E3792EE3540F20D101E4B3
:102BF000D2E730F60730F50320D101E492E6A3F0E6
:102C0000E3ACCCC006C007401D794DE3FE09E3FFED
:102C10007904E35438FA790CE3FB7903E3FC790295
:102C2000E330E733800CAA30530238AB38AC2F3096
:102C30007725E8541FB4010E796FE330E70853029B
:102C400030430220801179F6E354105302284202E7
:102C500079E7E3FE09E3FF796DE37002EEF309EF34
:102C6000F3D007D006EA20E41020E3047404800BBC
:102C7000EBA2E2440C92E080027400A3F0C2D17493
:102C8000405C4A03C4A2E072E192E1A3F0400F204D
:102C9000F10CE854E04401F8907CA0F0D2D1907C93
:102CA000A57C197D1BEC83600BFAED83F912F3B858
:102CB0000C0D80F1D320D10122D0E0D0E002AAFD9A
:102CC00006020501010100444177813347C375A025
:102CD0004D20D50820310B75A04CD3222031F8753A
:102CE000A04E22E4FD75A07C79BB90590F741012A0
:102CF000712CE030E003ED09F30DBD06F0B9BC0323
:102D00002009F322E8541F90AD0E9390AD2B730071
:102D100001040D10130104070A0D10130104160A13
:102D20000D10130104190D10131C1F1F2202AEDB1E
:102D300002B14702AD4D02AD6202AFBA02AD8E02E2
:102D4000B0FC02AD9702ADD702B99402A711907CF6
:102D5000B5E0600814F012AEAE08800118E8907C6F
:102D6000A0F022907CB7E0600414F080EC12AD5B20
:102D7000907CA1E0F5F030F308907CC2E0B4010152
:102D800022907CB6E004F030F0D8740C02AF829050
:102D90007CC3E060C402B301907CC2E0FD700D040E
:102DA000F012AB87907CB57401F080A2DD0B04F0CB
:102DB000907CC1E0907CC38016DDA1907CC3E07064
:102DC0000E7403907CC2F012B12D12AB8E80D5141C
:102DD000F07812790002B316907CC2E0B43003029E
:102DE000AD5BFD04F030E00512AB87800312AB8EC3
:102DF000EDC313FD907CBEE02D907CB8F002AD5881
:102E000012211720920CD2239067087401F0D3226C
:102E1000C3222023FB12AE3780F6E50F20E4082002
:102E200092EE12F81880E9309204D22480E2302425
:102E3000DFC224530FEF80EAC0A875A80075140004
:102E40009058FE12722A530FE0C221E4907CCFF01A
:102E5000907CC7F0907C9EE0907C9FE0907CA0E00E
:102E6000D221D0A82230230F904C0AE020D5052093
:102E7000E105D32230E0FBC322907CA0E020D509FD
:102E800030E709547F6005C32230E7F7D32275A8E5
:102E900000E0B2E5F075A88712ACCC7932E3B2E27B
:102EA000F330E2012212AE785004E0C2E5F02212C3
:102EB000B2B1907CA1E030E108907CBEE0FBA38041
:102EC0001230E40A740012B29CFBA3A380057B01BC
:102ED000907CACE0907CB7F0A3EBF022E824029069
:102EE0007CA0F0E4907CC9F0A3F012AF6AFCB406B9
:102EF0000040167D00907CA5ED12712CE06004FB73
:102F000030B4BF0DBD04EE801A907CA67403F0ECC3
:102F100090AF349360C590AF4A12AF76EC20E203D5
:102F200012B529EC90AF519390AF5912AF7690AF94
:102F3000EB740480420000050509094241525160CA
:102F4000434B34593D3D4860525A251B29301B28BC
:102F5000421B2A3C0101010301030F1B7D904C0C15
:102F6000E0C45407B40500B3922222A222907CA1AF
:102F7000E003C4540333226009FAE49312AF82A33E
:102F8000DAF822C083C082302215C0E0907CCFE006
:102F900004F0042582F582D0E0F0D082D083223084
:102FA000E7E8B4A00050E364C0C0E0907CCFE00448
:102FB000F0042582F582741BF080D112AD58907C0C
:102FC000B8E0F912AFF512B03412B0BC606630F759
:102FD0006312AF6AB40200405B740290AFEF12AFAD
:102FE00076EC2323540390AFF19380971B5B306DF5
:102FF0001B233536333412B28630D11CE8904AC5D3
:1030000090E703904B4AE0FCA3C083C082907CC54C
:10301000D0E0F0A3D0E0F022C00130E6011912B2F6
:10302000B1740812B28FE91475F003D00112B2A581
:10303000A3A3E0FC22907CA1E0F5F020D114907CC9
:10304000C0E0FDA320F110740312B29CFDA3A320E5
:10305000F4057D01907CABE0FBEC6003EB03FB200F
:10306000F155907CA4E020E14EC0F0C001C0048D79
:103070003BEB2D14F53C907CB9E0FBF8C00312B299
:103080008612B1CFAD01D0031BEBB53B00400A1255
:103090007E76E06D54F660F0A30B8B3BE53C0BB500
:1030A00003004007A3E06D54F660F1EBAD3BC39D18
:1030B000FBD004D001D0F0907CC4EDF022E5F054B8
:1030C00060C2D57002D2D5C0F0C00420F225EB2D2D
:1030D000F818C001C00312B28612B24EE9D003D074
:1030E0000120E30F5300DFB8000954F220D502702D
:1030F00002DBDBEB907CC3F0D004D0F022E824FDAF
:10310000407CA0F012B28630D10930E606E8A2E792
:1031100012EF91907CB8E004F0907CA1E030E20ED8
:10312000907CC2E030E0077819790002B316740D84
:1031300012AF82907CBAE4F0A3E0600612AF82E4A2
:10314000F022740A12AF822212AF6AFC12B18BEC29
:10315000B4020040F2790012B2BBBC0600402490D9
:103160007CB4E0FB907CA8E06B60057D0312B4BFEB
:10317000907CA5E0FB12B443BC07CC907CA7E0FB9D
:1031800002B443907CC9E060BE02B42078A012B1C2
:10319000AC907CA1E030E126E4F09060B8F0907C47
:1031A000CBE0907CA0F012B1BDB2D58011907CA094
:1031B000E0A2E792D5C858F022788012B1AC907C9A
:1031C0009E30D501A375A800E0543FF075A8872272
:1031D00030D105907CC58060740312B29CFBB500B1
:1031E000028005400302B247A3E0B50000405974D5
:1031F0000012B29CB5010280025025A3E0B5010087
:10320000801ED2D1740A12B29C6015FC740512B2F1
:103210009CC8C39B2C4005B500004002C3982BF806
:10322000C0D012B28630E60119D0D0740875F00310
:1032300012B28FE91412B2A512B292E81412712CD4
:10324000E0F8438380E0F922740675F00280E11211
:10325000B1CF907CA1E020E123907CA4E04954010F
:10326000601E907CA3E0601430E30330D112A2E032
:1032700054F659700B500574F2596004E930E106B8
:103280007820E9C2E1F922907CBAE0A2E792D1224B
:1032900012B29CE0C0E0A3E0F583D082222A9059CC
:1032A0001012712CE022A42582F582E5F03583F519
:1032B0008322907CB6E075F010A4FA22BC02004094
:1032C0000A907CCAE0C954F2B5010122F0F97403F6
:1032D00090AFEB12AF76E910E70E10E61010E51292
:1032E00010E414746D02AF82902B7E800D902B7AC7
:1032F0008008902B808003902B7CF9740212AF76AB
:1033000083D414F0A3E0F804F0907CB8E0F912B292
:103310008612B2B112B24E12AF6AFC12B53FC08330
:10332000C08212B2BBD082D083A905ECC313600D5A
:10333000FADA028038DA0302B3D202B3F5BB020430
:10334000E802AF82B901028003E493F8B823028057
:1033500014C083C08212B697D082D083400730E772
:103360000574208001E8A312AF82D9DD22BB0324BB
:10337000907CA6E0B40310907CC9E070067401F064
:1033800012B424E802AF827403F090AF4A740312BF
:10339000AF7680E3BB020512B41880E7B90105B827
:1033A000200280DFC083C082907CA6E0B4010A9036
:1033B0007CC9E06016C2D580447401F090AF4A74B5
:1033C0000212AF76744212AF8280E47401F012B43C
:1033D0002480E2BB010BC083C08212B418C2D58026
:1033E0001CBB0302808ABC040812B42853007F80EF
:1033F00092430080808DC083C08212B443D082D0BB
:10340000E4D908E8A2D592E702AF8209E493A2D5F5
:1034100092E712AF82A3D9F422907CC9E060F9E46C
:10342000F0740F801C740E8018748E8014748F805A
:1034300010741B12AF82747D8007741B12AF8274EC
:103440007C02AF82C2D5907CA9E0B82006600EE471
:10345000F080CE907CA512712CE0B5030122EC30F7
:10346000E011907CAAE0907CA512712CE0B50303DA
:10347000D2D522907CA5E0B50308907CA97400F019
:10348000809FA3E0B50308907CA97401F08096A307
:10349000E0B5030FBC06028090907CAA7402F0D2C3
:1034A000D5808EA3E0B5030FBC06028080907CAA75
:1034B0007403F0D2D58083EBF07D0312B4BF80E8B3
:1034C000741B12AF82BB020874282D12AF82805A7F
:1034D000BB0A1D907CB2E0700474288002742C2D0D
:1034E00012AF82907CAEE0FAA3E012AF82DAF9224A
:1034F00090B510E493B50311A3E4932D12AF82A30A
:10350000909360EB12AF8280F6A3E49370FBA380EC
:10351000E201284200032830002028253500212C14
:10352000410022283E0040283C00907CA2E0540F3D
:1035300090AF3A9312AF82B42505743612AF82224F
:10354000907CA2E0F5F0E97B017D0130E30302B558
:10355000E1B800028003B82003782022501318BC81
:10356000020040064300607B0322E890B6CF02B61B
:10357000A9B87F00501D30F70C12B697400420E721
:1035800004F87B0222BC02005008E5F0540F6002F0
:10359000782022B8A1005006E8945E02B6B130F758
:1035A0001312B69B50DBBC06005009E8949F90B7FD
:1035B0004D02B6A97B4020F615902C82E493600F53
:1035C000B50008BC060040E37B2122A380EE22AABE
:1035D00000D2D1902C95122CC74001F8B8FF027888
:1035E000FD22B8200302B5585004E802B6B1B87FF6
:1035F0000280F25011BC060040037B2222E8942096
:1036000032B7AD02B6A9B88300501E12B5CEBC04C5
:1036100000400C7B4030F6107B20BC06005009E8CF
:1036200094A090B6EE02B6A922B88500501530F7E6
:103630000812B69B400302B580C3E8948390B6CDD0
:1036400002B6A9B8A000409D53007F907CADE0FB7E
:10365000B4010302B584B40306BC0200403522B4B1
:10366000200930F616BC0600402922B4210520F6B8
:103670000A80F2B4220280EDB44008BC040040137A
:103680007B4022B40207BC040040F780D8BC06008F
:1036900040012278207B0122C2D18002D2D1AA002F
:1036A000E5F0540F122CABA802227B019310E70225
:1036B000F8227D02FA23B484005003430110B4B40D
:1036C0000040050DCA945A2A90B80B02712CD96695
:1036D0002A23898C8D8A6F2BA68B2B2B2B2B2B7E51
:1036E0003D2D3D5F2B2B2B2B7CC2C3C4C5232E212C
:1036F00063235F595FC64FDA61C75F5F5F5F6F2B00
:1037000073335F75C82E5F316FC9DBDC5F3F4141AA
:1037100041414141CA4345454545494949495F4EB3
:103720004F4F4F4F4FCB4F55555555595FCC61615A
:1037300061616161CD6365656565696969695F6ED0
:103740006F6F6F6F6FCE6F75757575795F5F2021C5
:1037500063234F597CC622DA61C77E2DDD2D6F2B86
:1037600032332775C82E2C316FC9DBDCDE3F414177
:1037700041414141CA434545454549494949444E6E
:103780004F4F4F4F4F784F5555555559CFCC6161DD
:1037900061616161CD636565656569696969646E6B
:1037A0006F6F6F6F6F2D6F7575757579D079D1D219
:1037B0002D28297C5B5B5D5D282829297B7D3E3C8B
:1037C0005C2F20203E5F5F5F5F3C3D3E53D361D462
:1037D0003A447646477E7E4A784CDFD53D50515F6D
:1037E000535F5FD657585963205E76267C7E6162B0
:1037F000636465666768696A6B6C5F6E207071727E
:10380000F0745F667778797AD75ED8764E555348EC
:103810005358455845544551414B424C42534854E6
:103820004C46565446464352534F5349444C4431F8
:103830004432443344344E4B53594542434E454D34
:1038400053424543465347535253555344543830DB
:10385000383138323833494E4E4C53534553485320
:10386000484A5653504450555249533253334443B7
:1038700050315032534543434D57535045503938DA
:1038800039393941435353544F53504D41504E42AF
:103890003C3D3E3D50693C3E53633C3C50723E3E95
:1038A00041454F45737361656F65546874682D7643
:1038B0007C2D3A2E6F4F3D3E567E3C2D2D3E696A43
:1038C000284329312F34312F32285229332F343CC9
:1038D0003D3EA23192D512AE675021C0A875A80016
:1038E0007514009058FE12722A303908530FF043B5
:1038F0000F08800630380312F822D0A89060B8E490
:1039000074A23192D5907C9EE054EEF9A3E054EE7F
:10391000FAA3E0FB7801500108E6E4F6EB541FB48B
:103920001A005009907CA1E030E113E4F0907CCBC8
:10393000E0907CA0F0630003E6C2E7F6800512AEDB
:10394000785029C22174D1907CD0F0E4907CCFF0E3
:10395000907CC7F0906048F0CB541FB41B00400C23
:10396000741B12AF82745C12AF82D221907C9EE9EC
:10397000F0A3EAF0A3EBF0E53930E20C5339BBE5F4
:103980003A5414600375468822BD1102D322BD1338
:1039900002D322C32212A301700302A56022904C1D
:1039A00001E020E23375A800A226400530312680D0
:1039B00003203121C24812EC8DE520F0B226A22668
:1039C00012EC8DE0F520904F99E0D2E4F075A887D5
:1039D000D214E4F51375A88722206B293072269043
:1039E0004C82E0B40105740C02743DB4021702006D
:1039F00024206B1130710E904C82E0B4020050050F
:103A0000070702743D12750D027310206B23904C52
:103A100082E0602014600BBD3517904C2BE0C2E3B0
:103A20008009BD410C904C2BE0D2E3F0780012FCF1
:103A30000D02750DBD25FA7402F02220779AB800A8
:103A4000010802DD29207790B800010802DD9A20E4
:103A500077E8B800010802DD812077DEB8000108B0
:103A600002DD42D265D266D262904C727406F002D8
:103A700073103096EE2077EB12F2A7904C82E05450
:103A800003FB12A4B5D2751273F202F2A72077D30A
:103A90003096D079013031027904904C01E030E267
:103AA0000109904C43E0B5010050B8EEB419005044
:103AB000B220790D79513060027929EFB5010050BB
:103AC000A2905901E0B506004099433708904C8216
:103AD000E0F812A54D0273F2207730904C81A3E0FC
:103AE0006019B4FE04740C8012C082C08390849765
:103AF000F5F0128C9AD083D082500D30E0033071F3
:103B00001F30E30854F64238D534D32254F65238E5
:103B100080F6904FA1E0040410E300F020E22B9027
:103B20004FA230E101A3E0F5F090F04DE0F4543FF6
:103B3000FC30F00590F049800390F041E0540460BF
:103B400003430C4030F00402BB9922904C01E0206A
:103B5000E20830E10C30E009800330E004431B133D
:103B600022904C00E030E311431B03301F0312BDD1
:103B70000DEC545010E43F8042431B10530C4FECAB
:103B800043F00220E10353F0FD203D03303C0520CB
:103B9000E002D2F412BD0D02BBC2904C01E020E263
:103BA0000830E10C20E009800320E004431B802260
:103BB000EC546010E50553F0FD8005440243F0022B
:103BC0004409FC30F703430C80904FA430F002A36B
:103BD000A312BE147003430C1030F314747530F04C
:103BE0000590F04A800390F042F090BE3802BC3657
:103BF00030F203430C20904FA830F002A3A312BE72
:103C000020E493A354C06001A3E4936CF4FCA3E408
:103C100093A3FB5CFC60147A08EC03FCEB13FB50F1
:103C200006EC20E70BA3A3DAF0802902BCE95005DB
:103C300012BE248002A3A3E582A883904FA830F08F
:103C400002A3A312BE2FE49330F004F51D8002F509
:103C50001CB4FF0AA3C082C08312BE24E47353F0D5
:103C6000F330F00790F04AE51D800B90F04230F4FD
:103C700003531CFBE51C20E407B48B07747580021A
:103C80007465F030F00FE51D20E105431B808024B2
:103C9000531B7F801F904C00E030E30FE51C20E1B8
:103CA00005431B10800E531BEF8009431B03E51CCB
:103CB0005403621B904FA830F002A3A312BE1FA3AF
:103CC00030F004E51D8002E51C54C0601D30E7069D
:103CD000E49378008008E493F853080F54F0904F71
:103CE000A430F002A3A3F0A3E8F020410C30F004CC
:103CF000E51D8002E51C30E20553F0DF800343F050
:103D0000D0C2F4E5F0904FA230F001A3F022EC30E5
:103D1000E64F101F31AA1EBAA500500FBAA00050DE
:103D200005BA4F005005431B048003531BFB203C86
:103D300003303D2D904C05E0FAEC20E204EAC4800B
:103D400001EA540F7006904C02E080082402F82328
:103D500023232328B51E0280087840FAF51E12445A
:103D6000C32220F005203C0F8037203E0A803220FD
:103D7000F003203D02802A02BDFEA23192D1904C78
:103D8000E0E020E10865F0A2E09231D32265F03056
:103D9000E0F5C32212BE086066800612BE0820E568
:103DA0005EC3805C12BD79505712715920310B539C
:103DB00046F920D1131273F2801453469F20D1F597
:103DC0001273F2904FA08003904F9F7401F002BDD8
:103DD000F312BD79502A12724820310C904D34E014
:103DE00030E611430F408013904E34E030E6054337
:103DF0000F808007A2D19231C38005A2D19231D326
:103E00005183D082A3A302BC2D30F0028003904CDA
:103E100004E054302212BE1A7005A3E014F004220C
:103E20001271358006E493F8A3E493F58388822227
:103E3000F0A3C8F08882F583220340403DBE83038F
:103E4000101043BE8007101049BE8047101251BEAB
:103E500051BEFF61BD7EBEFF6EBD65BEFFD0BD60C1
:103E6000BE0F2020EBBEA24710126DBE83BE230101
:103E70000172BE2F020379BE83BE23020283BE03FA
:103E8000020283BEFFA3BD88BE830710108EBE430F
:103E9000C1181896BE43BE0B11119DBE43BEFFD084
:103EA000BDA8BE8B071010A8BE0F202BD1BE43BEED
:103EB000B3BEDABEFF93BDA8BEFF9ABDC7BE8F00DA
:103EC0003838A8BE43BEDABE8F1E3838A8BE43BEFF
:103ED000DABE0B010BA8BE43BEB3BE0B4040DFBE33
:103EE0009B031010E5BE8B011010A8BE0B4040F0E4
:103EF000BE9B031010F6BE8B01101060BE008080C8
:103F000012BE12DB12904F25303103904F27E04450
:103F100002F0227B0212A4D812F29A12BF2B12E0F6
:103F2000767B0512A4D812F2A7021341904C41747B
:103F3000503079027484F012EF7412BF4F12BF0434
:103F4000904F26303103904F28E0D2E0F002A52CAC
:103F50007401904CE7F0A3F022904F25303103908C
:103F60004F27E04401F012A53780B6904C0075A0B1
:103F700051797E7B02780A12BFB1904C2B75A0510B
:103F8000796930310575A05179A97B0A780C12BF87
:103F9000B190517C3031039051BCE0A2E19279752F
:103FA000A04C792B904D2B303103904E2B7A0A0286
:103FB000F3B8E3FA09E06AFAE883085AFAE06AF02B
:103FC000A3DBEF2216088000C0FF3F000000008046
:103FD00012C17712C00012F3159051703031039066
:103FE00051B0E054F7F012724812B8D112F818121A
:103FF0007399127150530FEF12C00D12AE0202DB13
:1040000072E54754036006123153D2E7F022C2230F
:10401000906708E4F02212C088123E9D12ECAD7841
:104020001EE4121FF512A67A12BF6A12C1A91272FB
:10403000E712458C1245BC12EFF312A53712BF2BC5
:1040400090517EE05406F5F012D73A904F2530316A
:1040500003904F27E04402F0A3E04406F012F3156A
:1040600012C25812EF7412FC62904FA25003904F8C
:10407000A3E04408F012C09102BFEE12C08875F0B0
:1040800000123BEE12C1A2809F904C00E0904BF2D8
:10409000F022904C00E0F9904BF2E06920E401221C
:1040A00002A67A75F000123D2B12C1A212DB121289
:1040B0001A43021EFB531FFE123E7E70127A1875C1
:1040C000A07B791490519112F3B812FCB98003438C
:1040D0001F01800675F000123E2712C1A202DB12FA
:1040E00075F000123DC280F212FD07123E6080C5DD
:1040F00012739912F31512C00D12AE0212C1A91259
:1041000090FB90516B3031039051ABE0C2E1F090E5
:10411000516D3031039051ADE0D2E7F090516E30E7
:1041200031039051AEE0D2E0F090517C30310390F9
:1041300051BCE0541F44C0F090517B30310390518A
:10414000BBE0540D10E30444B2800244B6F0905C2E
:1041500081303103905CD6E05408F89051693031D9
:10416000039051A9E054F748F012458C1245BC1257
:10417000EFE712C25802DB12C275904F43E03031B4
:1041800004D2E18002D2E0F02212B8D112F8181263
:10419000F332C275904F43E0303104D2E38002D253
:1041A000E2F022904BCF7401F02212C188C26CC29F
:1041B0006E5337AF12889D1288420285FF7B001232
:1041C000A5AC128911904F43E4F012F27DA2313375
:1041D000904F8CF012C23012C27712F29AA231E4E0
:1041E00033FCA226923192E05401FD12EA5375A0ED
:1041F0004C790090517E7A1312F3B875A04D792B4B
:104200005951697A1412F3B875A04E792B9051A9BF
:104210007A1412F3B8C20012C2E37C087B0012A425
:10422000997C04C26412A3DC12C9F912E74A02594C
:104230005030770312C246904E02303103904D0247
:10424000E030E73312EADC12C26AC27702F00D9066
:104250004C2DE030E50312EF58904F95303103902C
:104260004F96E06012127399E480027401904F95AA
:10427000303103904F96F022533ADD2031333073C2
:1042800003433A02904E02E030E303433A20904F5A
:104290008F12EC48904C2EE0904FACF0904E4D12A7
:1042A000EC57904F9212EC48904E2EE0904FADF0AC
:1042B00022307303433A20904D02E030E303433A47
:1042C00002904F9212EC48904C2EE0904FADF0903F
:1042D0004D4D12EC57904F8F12EC48904D2EE090C0
:1042E0004FACF022904F447E007F007D18EEF0A38B
:1042F0002484FEEFF0A33400FFE4F0A3DDEF2212EC
:10430000E510907FF9E06007E4F07B8012A60B12C5
:10431000DAACC22EC24A304D03121E66C24DC24BE9
:10432000C24C1260C412C53312C55D7B0112A5AC2C
:1043300012F29A12EC96904C2B7A1412F3B81241A6
:104340002812C5FF904F8CE020310520E008800343
:1043500030E00312EADC12891112FC7012C3CD2086
:10436000310812C60612C60D800612C61412C618EF
:1043700012C3D912C3B212EADC12C3CD2031081223
:10438000C60612C60D800612C61412C61812C3D96C
:1043900012C3B212F29A12F27DC22F123ED212C78B
:1043A000F430480C905F32E0B4400302F242C2485D
:1043B000025950207517207314307011904F9530AA
:1043C0003103904F96E06005E4F012EF1122904F18
:1043D0008F303103904F9202EC57905FC23031031F
:1043E000905FC3E0904C0330E003904C07E0F8206E
:1043F000E30974FB30310274F75247E85407702523
:104400003046203111202602C203540F6017534654
:10441000F8434608800F302602C20354F06006536A
:10442000468F43468012F9D412A47712A48612A5AF
:10443000C712A50012A495C204904C2BE020E505FC
:10444000207D02C26F904C32E0A23192D520E2056D
:1044500012AEA4800312AEA31283EE307816904FF2
:10446000AC303103904FADE0F9904C2EE06930E470
:104470000312C7A0904C2BE030E54B9051693031CE
:10448000039051A9E030E56C12C80D12F315C27506
:1044900030730312C677740380777405807312C576
:1044A0002A30E240740420736890516930310390DF
:1044B00051A9E0FB904C2BE06B5407B40404740842
:1044C000804F7403804B9051693031039051A9E0C3
:1044D00030E5CB12C80D3073CB12C67712878C1221
:1044E000DBCC80C012C52A30E0143073AD20E40765
:1044F0007406801DE4801A12C80D74078013FBE453
:1045000078730AC275EB20E4EE7402800430750102
:1045100004FB904F43E0203108A2E372E092E08078
:1045200006A2E272E192E1F002A5A4904F43E030CE
:1045300031010322904C0075A051787E7D1312C585
:1045400051904D2B78697D1412C551904E2B78A94E
:104550007D14E2F9E0C9F069F208A3DDF522783BA9
:104560007906E4F608D9FC90C59A75A051E493B495
:10457000FF028018F8E2F9740193596009740293FC
:10458000F974039347F7A3A3A3A380E1904F237883
:104590003B7D06E046F008A3DDF9227F043B018065
:1045A000FF3B0281203B02820F3B0284FF3B0485DC
:1045B000203B04860F3B048AFF3B0890023B107FA0
:1045C000033B207E083B408F303B408FC03B8069DF
:1045D000073D80A9073F806AC03D20AAC03F206EEA
:1045E000083D40AE083F407C013D10BC013F106BD0
:1045F000203D08AB203F087C1C3E08BC1C4008FF47
:104600007923790002C61C7825790802C61C782611
:10461000791002C61C782780F0782880F374082966
:10462000F975A04FE210E706236002D9F822F2C024
:1046300000C001E990C63D127141D001D00080E177
:1046400085C669448044AFF7D5C70FC71A73247372
:1046500070C675C600C74EC2A0C7E2366BC77AC720
:1046600067C689A609C7E0C712376612378602F304
:10467000CC7B0102A5B8E4F27B0012A5B812FDE7DD
:1046800012C7E002475DC211E4904F98F0904F9935
:10469000F012C732904C01E030E21212C713D21D63
:1046A000E4904F8EF0904F8DE0F520D214C226C2D8
:1046B0001DE4904F8CF0906001F012F332904F2582
:1046C000E04406547FF0A3E04402F0A3E044065423
:1046D0007FF0A3E04402F0904CE77401F0A3F09067
:1046E0004DE7203103904EE7F0A3F0E4904F95F0B2
:1046F000904F96F0904AC57A8512EF797A8502EF4D
:1047000010123F3612C77A02DBD0123F3602DBD0DE
:1047100012C732E830E11B540104F812314DB411D4
:10472000005003E4F0227410F0905F44F0905F2397
:10473000E8F022904C01E0F812C759F990517FE05F
:1047400068F812C759B4030122B40107B901012264
:10475000027324B902012202731A20E20620E10347
:1047600074032220E003740122740222904F43E07C
:10477000303104D2E58002D2E4F02212C18812FC6A
:10478000201289E412C25820730FE53A2031042028
:10479000E1042230E5FC02BF0412878C12DBCC80DE
:1047A000F5904C2EE0A2E4904C4478082078133029
:1047B00071107910E983307803400123F009A3D800
:1047C000F322791880EE010140400002014001010E
:1047D00001010000010112718FB23112718FB231EB
:1047E00022A231904BF4E04004D2E08002D2E1F00A
:1047F00022A22680EE904BF4E020310410E0052246
:104800004DE10122F02075FB2073F802DCC412B8E0
:10481000FB02F8180D6E6F7420636F6E6365616C38
:104820006564FF07616666696368E9FF0365696E31
:10483000FF0B3C436F6E6365616C65643E2020FF37
:10484000073C63616368E93E202020202020FF0CA4
:104850003C756E73696368746261723E20FF907F7D
:10486000F9E06063BB005FEAB4F217E4F0907FFA0E
:104870007480F0FB12A60B7B0512A4D812F2A702DB
:104880001341B470004009B47A00503A540F8021AB
:10489000B46C047410801AB46D04740E8013B46E7A
:1048A00004740F800CB45000401CB4540050179492
:1048B00045FB90E795E0B40105BB07005008907FE9
:1048C000FAEBF002A60B22EABB0119304D03021BE2
:1048D000DCB4090F90E787E0B40A08E53FB40703AA
:1048E00002DA6722B4F20302D25CB42909204D0334
:1048F00002D25C021BDC20E645B4121412C9EC3073
:10490000D203121E6612C9D81220AC1220C38056E0
:10491000B4131412C9EC304D03121E6612C9D8121A
:1049200020AC1220C38052B4143512C9EC304D03B0
:10493000121E6612C9D81220AC1220C38062B44184
:104940000302CF87B4420302CFBBB44406204D0C10
:1049500002CFD6B44309204D0302D1A7021BDC309D
:104960004D03021BDC2290E787E0B4000122D25500
:1049700090E7877400F002CA2990E787E0B4000D41
:1049800090E795E0F8740BB8004604804314B40631
:104990003FF5F090E795E0B4020215F0E5F08030C5
:1049A00090E787E0B40C047400802504B4060BF58E
:1049B000F090E795E0B402168012B40C13F5F09075
:1049C000E795E0B4000280067400800405F0E5F08D
:1049D00090E787F0C25202CA2990E787E0B4080C3A
:1049E0009087BC7D50E05420F0A3DDF92290E7874A
:1049F000E0B40A05C24B0289112290517EE05406B0
:104A0000CEE7FE90E7DDE070FDEEF075350090E753
:104A1000877400F012CB02E490E78EF090E782F00A
:104A2000904CC8F090E792F0F52A9000007B607EF1
:104A30000DE4F0A3DBFCDEFA12CB0290E787E0FE88
:104A400075F030A42400F53DE5F034CDF53E7B0251
:104A500012A4D812DA9312D593C2D112DB2ED2D17E
:104A600012DB2EEEC24EB4040890517F12FC659208
:104A70004E90E780E533F090CF6EEE93F533753FBF
:104A800000E53F12D7EDF5A075400012DB16E53FBB
:104A900023253DF582E4353EF583E0F53BA3E0F5C3
:104AA0003C740012D76D23F5F005F090CAB893C599
:104AB000F093F58385F082E47328CB17CB28CB28BD
:104AC000CB28CB28CB5FCBEDCBAECCBCCCB6CCD4FB
:104AD000CCD8CCB6CCE0CC11CD1ACD28CB28CB2865
:104AE000CBB6CC30CD70CD7FCD98CDBECDC1CDD0A5
:104AF000CDC8CDD5CDDBCDE7CDFECD23CE27CE5055
:104B0000126DCE90E78EE0B40C0412A6752290E7E9
:104B100087E0B40CF802A67090E795E0B40002803C
:104B200008053312DB1602CE7512D785741F12CF1B
:104B30003812D8212403305602240412D7BB740142
:104B400012D76DB4140302CE75743712CF387402C5
:104B500012D76D12D8092403305602240402CD2A3C
:104B600012D785C37B0112213C50027B0812DB2146
:104B70009051723026039051B2E030E72690517E7A
:104B8000E090C84E20E20990C83F20E10390C83071
:104B9000E493C002FAA3E4937B0112DB22DAF6D09D
:104BA00002803712ECCCE0B41F00502E6025C0020A
:104BB000FA75F00AA3E07B01C083C08285F0838888
:104BC00082121D80A38583F0D082D08312DB22DA8B
:104BD000E3D00274157B0112DB227484C39540FB81
:104BE00012DB2102CE75B407004002E4F02212D796
:104BF00085745012CF38904BE07401F012211EE002
:104C000012CBE5A3C002FAE5838582F012CC84744E
:104C100015F0905C96303103905CEBE012CBE5FA36
:104C2000A3E5838582F012210DC0E0741812712C67
:104C3000D0E012CC877415F07402904BE0F0122192
:104C40001EE012CBE5FAA3E5838582F012CC8474D2
:104C500015F0905C9D303103905CF2E012CBE5FAE8
:104C6000A3E5838582F012210DC0E0741812712C27
:104C7000D0E012CC877415F0D002904BE0E4F075D0
:104C8000404F02CE7512210DC000C001F9A8F0EA14
:104C9000600E12CCA5E012CCA4F0121D80A3DAF2B3
:104CA000D001D00022A3C8C582C8C9C583C92212B9
:104CB000D785742A12CF3812D78502CE7590E79522
:104CC000E0B4020405338008B4000280E212D78504
:104CD000053302CE75D24F80DED25B121EFB02CEB0
:104CE000B112D785740912CF38741912DB1712DA92
:104CF00006C2516009F5F02325F0FB12DB21745B3D
:104D0000D7DB17745D12DB17743912CF38741902B0
:104D1000CE7215401812DA3602CE7512D785741F7E
:104D200012CF3890E78912D85A240312D7BB02CE8B
:104D30007512D78590E787E0B40417900035744367
:104D4000F0A3746FF0A3746DF0A3F0A3E4A24E344B
:104D500031F0743C12CF38740012D78990E795E097
:104D6000A2E090003F74349400F0A37430F002CEBF
:104D70007515401874127B8412DB227F8402CE7872
:104D800090E787E0B4000302CE75B4030302CE754A
:104D9000B40B0302CE7502CEB1740112D789741F11
:104DA00012CF38740212D78990E787E0B40B030260
:104DB000CE75743712CF38740312D78902CE7502BC
:104DC000CEB112D78574118002741612CF3802CC7E
:104DD000B612D78580F312D78502CE7590E7DDE055
:104DE00070FD7404F002CEB1904CC7E0FB90E7DD9B
:104DF000E070FD0582EBF015827405F002CEB11271
:104E00000085740A12CF38904CC7E0FBB40A0050FA
:104E10000812DB16EB24308008743112DB17EB2408
:104E20002602CE72740A80A3740912CF387401125C
:104E3000D76DA2E092D1740D30D102740E12DB173F
:104E400074127B2F12DB22740C30D102740B02CE51
:104E5000721815407D083079027D0D740412D789CF
:104E6000DDF9307911743112DB177432800512D7F5
:104E70007E800312DB17854007E53FFE0EBF8400EE
:104E800050010F305409BF500050107F50800C204B
:104E90007909BF5002800440027F5012A4267B048F
:104EA00012A4F990E787E0B40808E53FB4110312B3
:104EB0001A43C251C256C257053FE53FB41802809B
:104EC0000302CA8090E780E0F53320545B90E787C7
:104ED000E0F890E78EE0C8F0F5F090CF479390E7C8
:104EE0008FF0E5F090CF5493F9E5F0B4010A90E724
:104EF00095E0B4000F09800CB4050990E795E0B483
:104F0000B4020909E990E790F030550FC255E8B4B2
:104F10000700B392521490CF7B8007C252E5F09005
:104F2000CF6193F53F02D484C25490E782E0F53F0D
:104F300012D7DD85F03BF53C22F5F0C3954028F80B
:104F4000500205A085F0402203050505050505056D
:104F50000505040503110B0B1214110B110F120799
:104F6000101003050505050505050C0504050307D7
:104F700020293140506068768190959F0304050692
:104F8000070803040506070812D1914049E412D727
:104F90006DD2D190D39D02D5C6C250904BE0E0C0F7
:104FA000E0121E66D0E014904BE0F08003121E6603
:104FB00002D0E4128911C24BC25280F412D19C403B
:104FC00015E412D76DD2D190D3C502D5C6C2500216
:104FD000D11CD24D80F922E412D76DC2D190D3ED0D
:104FE00002D5C6E53FB405139051693026039051B0
:104FF000A9E05407B40404E01414F002D93DE53FDD
:105000000B05139051693026039051A9E05407B461
:105010000104E00404F002D92D02D92D90516C3026
:1050200026039051ACE0540FB400012202D93D9008
:1050300051723026039051B2E020E706122071022F
:10504000D93D2212D04F4005700312D07702D93DCE
:105050009051693026039051A9E05407B4040280AE
:1050600003B4061290517B3026039051BBE0F5F05B
:1050700003035403C322D322E5F0D2E3C2E2F022B9
:1050800012D04F4005600312D07702D92D2052056F
:1050900012D19140EAA252B3925230520E02D0E4A1
:1050A000904CC8E0602314F0121EFB02D465904CB3
:1050B000C7E0601514F002D2E790E791E0600514B4
:1050C000F002D465128911C24B02D0E212DA0660F6
:1050D000AE1412D20712D21912D2307B0312DB2186
:1050E00002D253D252153FE53F12D7DDF58385F04A
:1050F00082E0B4140050EEB4091290E795E0B401D8
:105100000120D105C25202D4652052D9B40E0BE55C
:105110003F24F212DA0B90E792F002D465053FE5E6
:105120003F12D7DDF58385F082E0B4140050EEB471
:10513000090490E795E0B4010B20D105C25202D4D6
:10514000652052D9B40E0EE53F24F212DA0B90E737
:1051500092F002D465B40F0D90E791E4F012891833
:10516000D24B02D465B40B07904CC7E4F08020B456
:105170000604D24D8019B40716904BE0E070047419
:10518000018008B40109121E667402904BE0F0021F
:10519000D46590E78FE0B53F02D322C32290E79019
:1051A000E0B53F02D322C322E412D76DC2D190D41E
:1051B0001502D5C62230520612D19C500122A252AD
:1051C000B3925230520302D46502D11C90E795E0AD
:1051D000B401E202D11C22904CC8E0B40E012204BA
:1051E000F0121EFB02D465904CC7E0B40F012204FC
:1051F000F002D2E790E791E0794F3079027983B5F8
:1052000078012204F002D465C5F045F0305103C4A2
:10521000C251F0E5F090E792F0222325F0FEE53F41
:1052200012D7EDC8240AC83400C82EC83400F5A02F
:1052300022745B12DB17745D02DB1712DA06B40FFF
:1052400001220412D20714F5F012D2197B0312DBEB
:105250002112D23012D5E412A67002D465E412D71E
:105260006D90D43D02D5C674013052010412D76D41
:1052700002D62D90E78912D85A045401FC90E78990
:1052800012D8DFEC02D94B2290E791E0700122FFA7
:1052900075F00884ADF090501530260390505A25D3
:1052A00082F582E43583F583E0BD000280058D043C
:1052B00003DCFDA2E0B392D192E0BD0002800323A3
:1052C000DDFDF07D5420D1027D00E53FFAFB12D7D1
:1052D000EDC82FC83400F5A0EDF2EFF8F9AF3B753B
:1052E0003B0012A5E38F3B22904CC7E0FE90E7DD28
:1052F000E070FD0582EEF015827405F0EE75A005F4
:105300008C32B40A00500812DB16EE243080087488
:105310003112DB17EE242612DB1775020A75030A19
:1053200075000A75010D753B0012A5E3E490074274
:105330007D2FF0A3DDFC9007C67D2FF0A3DDFC9050
:10534000084A7D2FF0A3DDFC740012DA0BFD232D3B
:105350002442F582E43407F583745BF0A3745DF0B6
:10536000740112DA0BFD232D24C6F582E43407F50F
:1053700083745BF0A3745DF0740212DA0BFD232DCD
:10538000244AF582E43408F583745BF0A3745DF07D
:105390007A0E7B10780A793912A5E302D465E4D03D
:1053A000E4D0E4D0E4D0E4D0E4D0ACCF98CFE4D0E3
:1053B000E4D0E4D0E4D0ACCFE4D0E4D0B2CFE4D0B9
:1053C000E4D0E4D0E4D01CD11CD11CD11CD11CD120
:1053D0001CD1D5CFCCCF1CD11CD11CD1D1CFD5CF96
:1053E0001CD11CD1D5CF1CD11CD11CD11CD13DD975
:1053F0003DD9E2CF3DD93DD92ED07ED07ED08CD0C4
:10540000F0D08CD09FD0DC1BADD0CBD0B8D072D236
:105410003DD942D01BD02DD92DD9FDCF2DD92DD995
:105420002ED0B3D1B3D1B4D1CBD1D5D1D6D1DC1B11
:10543000E6D13AD2F3D172D22DD97FD01BD02DD95B
:105440002DD9FDCF2DD92DD92ED086D286D266D298
:1054500066D266D286D286D286D286D287D272D2DF
:105460002DD97FD01BD0907FF3E070FD12D59390A3
:10547000E786E0601090E782E0600A8F01AF3B753D
:105480003B0012D577E53F90E782F0700122F502EC
:10549000F50312D7DDF53C85F03BE412D76D90D4CF
:1054A000A302D5C6DAD4DAD4DAD4DAD4DAD4DAD4A8
:1054B00021D52DD5CBD4CBD4D6D4E8D4E0D4F9D4CF
:1054C00008D518D5DAD4DAD4DAD4DAD47D2679003E
:1054D00030526B79298067C25280F17D4F7900800C
:1054E0005D90E786E4F0021AB7904CC8E07D03B403
:1054F0000A010D90D5D593F98044904CC7E023F56F
:105500007525F004F97D03803590E792E0F5F023EE
:1055100025F0240AF97D02802590E791E0F97D01CC
:10552000801C7D1F791512D53DC24F021AB712D4C7
:10553000DAC24FD24D021AB790E786E4F022E53F77
:1055400012D7EDFEE990E783F00582C828F9F0054F
:1055500082EE34002480F5A0F00582EDF0FEE3B287
:10556000E5F309B9000205A0DDF4EE2814F501AF5A
:105570003B753B0090E782E0B40E004011B411008F
:10558000500C90E787E0B40C0512A5E3800312D617
:105590000B8F3B2290E786E0602C90E782E060264C
:1055A0000582F502F503E00582F500E00582F9E0E9
:1055B0000582F5A0E0FD2500FF1FE3B2E5F309B980
:1055C000000205A0DDF42223F5F00493C5F093F565
:1055D0008285F083E4731316191C1F25282B2E34A3
:1055E000373E414447904CC7E0FA90626C12712CF0
:1055F000E0C4540F23CA90625C12712CE0540F2A4D
:105600004FF00384C4FAE0540F4AF022907FF3E095
:1056100070FD90E7DDE070FDA3EAF0A3E8F0A3C31E
:10562000E99804F090E7DD7406F0E070FD22B40C18
:1056300000500A0490E787F0C25202CA2924F4906D
:10564000E78DF023F5F012E74AE5F005F090D6601B
:1056500093C5F093F58385F082E412D65F02E76C80
:1056600073EFC0A5D601BFA0D6CFBFABD689342E6D
:10567000D7A5349AD6681FD3C0611FA2C0D2D6D690
:10568000D6E7C067D764D758BFB0D69AD69AD69A0D
:10569000D69AD60BD70FD7B6D69DD602D8C602A6B5
:1056A0002CD25502C07A12DAAC02C0DFD25502C049
:1056B0001512E07602BF12907FF974FFF0904F252B
:1056C000303103904F27E0D2E7F0907FFAE4F0FB0F
:1056D00002A60BC2D18002D2D17D10905015302687
:1056E0000390505AE4F0A3A2D192E0F0A3DDFC7441
:1056F0000712D7EDF5A012DA367A077B0778007922
:10570000223079027983753B0002A5E3C2D1800281
:10571000D2D190E789E05477700122F5F0A2D192BE
:10572000F3E4A2F6C2F692E0907FF4F002417490A6
:10573000517E12D750904C0012D75090E7DDE070A8
:10574000FDE5F0D2E7F012D593D25412CA29021324
:1057500041E0F5F053F0F954062402B40601E4C523
:10576000F045F0F02202A67A12C0B402D2E7853BDF
:1057700082853C832582F582E43583F583E02274BB
:105780000112D76D8004E5330533F5F07401FB9009
:10579000E7DDE070FDA3E5F0F0A3E540F0A3E53F11
:1057A000F0A3E4F090E7DDEBF090E7E1E060FDFBD3
:1057B0002540F540EB28F8500205A02212D76DC213
:1057C000D1B41902D2D1F5F0740212D78D30D10DB7
:1057D00090E795E0700718187434F2080822232522
:1057E0003DF582E4353EF583E0F5F0A3E022F5F0E7
:1057F0002325F02444F582E4344FF583E0A3F8E058
:10580000F0900052E0F45401F022740112D76D20A0
:10581000E70B905C81302638905CD68033905CAB8F
:105820008016740112D76D20E70B90516930262045
:105830009051A9801B90517E304E15F5F0E53FB494
:105840000C02800AE5822404F58250020583E5F00B
:10585000543F2582F582E43583F583E0FDC083C0A3
:105860008290E7DBD0E0F00582D0E0F0740212D73E
:105870006DF5F0304E09E53FB40C02D2F5E5F05479
:105880007053F00F6006C4CD03DDFDFDED30F30471
:10589000540F801030F2045407800930F10454038F
:1058A00080025401FEE412D76DB4040B90517FE0E6
:1058B00020E204D25615F0EE2290E7DBE00582FEEE
:1058C000E0F5838E828019740112D76D904D2B30D4
:1058D0002603904E2B543F2582F582E43583F583D1
:1058E000E0FDAE82AF83740212D76D8E828F83F596
:1058F000F0304E09E53FB40C02D2F5E5F054705398
:10590000040FC4FF6005CD03DDFDFDED30F304544D
:10591000F0801030F20454F8800930F10454FC8017
:105920000254FE2CBF0002800323DFFDF02212D8B8
:1059300021C5F0B5F003E4800FC5F004800A12D849
:10594000217004E5F0800114FC12D8B8E53F12D7AD
:10595000EDC8241FC83400F5A075401FECC0E0243A
:10596000033056042404C25612D7BB7437C3954083
:10597000FB12DB21E53FF502F503781F7937AF3BDA
:10598000753B0012A5E38F3B740212D76DD0042043
:10599000E70122740112D76D20E60E904C2B30E700
:1059A00003904C0012D8D4804F543FB4120479288D
:1059B0008010B4110479278009B41304792F800270
:1059C0007930740212D76DF5F0547053F00FC4FFA4
:1059D000FDE7600303DDFD30F30454F0801030F286
:1059E0000454F8800930F10454FC800254FE2CBFAA
:1059F0000002800323DFFDF7740212D76D540F24D9
:105A00009012D76D02D62D740112D76DC25175F068
:105A1000006002D2F4B40102D251904CC7E025F0EC
:105A2000245CF582E43462F583E0305101C4F5F082
:105A300054F0C5F0540F2290501530260390505A60
:105A40007D10D2D17C08E0A3F5F0E430F00274546C
:105A500012DB17E5F003F5F0DCF0DDE830D108C229
:105A6000D17D017C0480DF227D4F3079027D8390DF
:105A7000E791E0B505012204FC249CF582E434039F
:105A8000F583E0B40006A30CECB505F690E791ECC5
:105A9000F002D46590E787E0B4020412DAB422B4CD
:105AA000030412DAD022B4090312DAEB2212DAB4B8
:105AB00012DAD0803790516C3026039051ACE0540C
:105AC0000F700D90517C3026039051BCE0C2E0F085
:105AD0002290517FE020E21390516A3026039051CA
:105AE000AAE054C0B4C004E0C2E6F022905169308C
:105AF00026039051A9E05407B404028003B40612AF
:105B0000F0517B3026039051BBE030E305C2E3D275
:105B1000E2F02202198022E4F2080540B8000205F2
:105B2000A022E4F2080540B8000205A0DBF52290AF
:105B3000E78720D10390E78EE023FA0A90DB929367
:105B4000CA93F5838A82E4936048A3FDAA82AB835B
:105B50008A828B83E49312D7ED2480FC8A828B8324
:105B600074019328F8E43CF5A0740293FC74039349
:105B7000F920D103E9F4F9E220D10359800149F277
:105B800008B8000205A0DCEFEA2404FAEB3400FBBD
:105B9000DDBE22B0DBB0DBB0DBB0DBB1DBB0DBB055
:105BA000DBB0DBB0DBB6DBC7DBB0DBB0DBB0DBB080
:105BB000DB000115151F1004111F07101137071006
:105BC000121F0710123707100107008420D25780D8
:105BD00002C257904C01E030E20D30310A90614A28
:105BE000E4F090614BF022A2E292D15003E48008ED
:105BF000904C00E023235403FA90614AF090614BEB
:105C00000712E738904C42E09061223031039061F6
:105C100022F020570690614D740CF090591F3031DE
:105C20000390594F7402305707E0A2E7740292E7DD
:105C3000F0780230D112780490592F74023057074F
:105C4000E0A2E7740292E7F074102582F582E4F096
:105C5000D8F690612030310CE0B403004002E4F04B
:105C6000906144E4F00582F090610130310390616D
:105C7000257418F0906001E090614EF0C25012E47B
:105C80007612E48220500E7B01740012E4D8740274
:105C900012E4D8800612E25812E28F12E19E12E15D
:105CA000B312E45B12E53BB23112E563B25020500F
:105CB000CD30D1089067847401F0800312E58B1217
:105CC000E65102E741202F0D20770A90590FE0207E
:105CD000E004207C3822307B199061003031039041
:105CE0006124E0B50602800A50230582E0B5060073
:105CF000401B307A34906102303103906126E0B568
:105D000009012250080582E0B50700501C9067F891
:105D1000E06009A23192F065F030E00D904F99E01B
:105D2000D2E0F0904F9A7401F022C00012A65512F2
:105D3000E1C5D000740012E4CE146023C25312DD1A
:105D4000D6802AC00012A65512E1C5D000741820D2
:105D50007304904C42E0FA740112E4CEB5020302DF
:105D6000E741D25312DDDF740012E4CE28FBC250AB
:105D7000D251906150E8F0740012E4D812E1B302FD
:105D8000DE13C00012A65512E1C5D000740212E461
:105D9000CE1460CBC25212DDD68029C00012A655A7
:105DA00012E1C5D0007450207304904C41E0FA74A5
:105DB0000312E4CEB5020050A6D25212DDDF740207
:105DC00012E4CE28FBD25090614FE8F0740212E446
:105DD000D812E19E02DE13C398500328F8E404228F
:105DE000285005EAC39BF822CA9A500228F82212CA
:105DF000A65512E13E12E1C5C250C25112E1D14096
:105E0000E2E52A54036039B4030AC25412E1CB120A
:105E1000A651802C30501190614FE0B40A0050EA36
:105E20007B022052120B800F906150E0B4030050AF
:105E3000D97B002053010BFAC25412E1CB12A610F9
:105E400002E741904F9BE0F5F0A2F7E492E0906109
:105E50004EF0A23192E765F030E707C0F012EADCBD
:105E6000D0F012E1C5E5F05407701B740012E4CEC7
:105E7000B4010302DF2312A655740012E4E21B1CD6
:105E80007401C0E08025B401357418207304904C6F
:105E900042E0FA740112E4CEB50200505A12A6553F
:105EA000740012E4E20B0C7400C0E0740012E4EF22
:105EB00012E2F412E40912E43412E3DA805AB40371
:105EC0001A740212E4CEB40102805912A65574026B
:105ED00012E4E21B1C7403C0E0802CB4024920735E
:105EE00006904C41E0800774503079027484FA7453
:105EF0000312E4CEB50200502B12A655740212E430
:105F0000A60B0C7402C0E0740212E4EF12E2C61297
:105F1000E35F12E41B12E3F1D0037A01C25412E1F1
:105F2000CB12A61002E7419061203031039061440A
:105F3000B40406E060EE148018E0F5F0C082C0837F
:105F4000904C3FE014D083D082C5F0B5F00280D4ED
:105F500004F012A655C25412E1CB12A65180C5908E
:105F60004C00E020E7012212A64D12E13E12E53B73
:105F7000904F9CE0F5F090614DE020F019601A140C
:105F8000F07B0012E1474007904E42E0FA80027A2F
:105F900018906125801DB418057B8002A62204F0AC
:105FA0007B0112E1474007904D42E0FA80027A18E7
:105FB000906101E0B502070B0B1582E014F0C003FD
:105FC00012E738C251A2319250C2317E007F618007
:105FD00006D2317E247F6112E56312E48212E25818
:105FE00012E1B312E45BB2512051E6A25092311299
:105FF000E563C25412E1CB12E741D00302A622129C
:10600000F04D12E13E90614AE0B4020274FF04F9DF
:10601000F00303F5F0904C00E0543F45F0F0C25718
:10602000800312EADC12E73812E47612E48290610F
:106030004AE06024B4010812E19E12E41B8022129F
:10604000E28F12E19E12E1B312E41B12E45B7400D2
:1060500012E4E29B400E800912E25812E1B312E40E
:106060005B12E1D112E741B2572057B6D25412E188
:10607000CB12E74102A5B012E1C512E48212E28F11
:1060800012E2B312E2C612E32512E34212E35F12F8
:10609000E41B12E3F102E741A22692F0906001E0D6
:1060A00065F030E014E43390614EF0904BD3E4F0AF
:1060B00090614AE0600612A64502134112A64D12F5
:1060C000C7F012E738D25412E1CB12A6491213419D
:1060D00002E74112E13E12E1C5904C42E0F5F0F9D1
:1060E000742212E4CEC5F0FB742212E4D87420129C
:1060F000E4CEA4F5F0740012E4E21425F0CB1425EC
:106100001289F084C9C5F0CB84B501050BC2558056
:106110000ED2557B01904C43E030310224FDF974DE
:106120000012E4D87420890312E4D812E1B312E417
:106130005BC25412E1CB30550312A5B002E7419087
:106140006001E090614EF022A23192E065F030E013
:1061500005207310C322904D2B4003904E2BE0542A
:1061600007B404F0D32212A65512E1C512E13E1283
:10617000E482904C41E0B45018740312E4CEB45160
:1061800040400E741E12E4CE74519BFB740212E464
:10619000D812E19EC25412E1CB12A69302E741123B
:1061A000E2B312E2C612E32512E34212E35F12E405
:1061B0001B02E3F112E27C12E2F412E3B712E409EB
:1061C00012E43402E3DA12E73802E47612E58B02D5
:1061D000E64E307A31740212E4E2C252906149E034
:1061E00090614FB503005006C3CB9BF0800ECCB539
:1061F00004005012D252C3CC9CF02BFBD25074023C
:10620000B4E4D812E19E307B31740012E4E2C25350
:10621000906148E0906150B503005006C3CB9BF0FD
:10622000800ECCB504005012D253C3CC9CF02BFB93
:10623000D251740012E4D812E1B3307C15904C4373
:10624000E090612030310524FD906144F5F0E0B527
:10625000F002C322E5F0F0D322740012E4CEFA7407
:106260001F12E4CE2A14FA904C42E0B502012250EB
:10627000FDC39B5001E404FB740002E4D8740012D7
:10628000E4CEFA741F12E4CE2A14FB740102E4D89F
:10629000740212E4CEFA741E12E4CE2A14FA904C60
:1062A00041E0B502012250FDC39B5001E404FB74A0
:1062B0000202E4D8740212E4CEFA741E12E4CE2A6A
:1062C000FB1B740302E4D879007A0030310B906133
:1062D0004AE0B4010479947A01740212E4CE147590
:1062E000F00A30790375F006A4C999FBEA95F0FC31
:1062F000740402E4EF79007A0030311490614AE0CE
:1063000006020D90614DE075F014A40404F9AAF0A2
:10631000740012E4CE1475F014A4C999FBEA95F048
:10632000FC740602E4EF2031012290614AE07B0018
:106330007C00B401047B947C01740812E4EF740CBB
:1063400002E4EF90614AE0B4010D7B907C013031B2
:106350000A7B247C0380047B207C03740A02E4EF24
:1063600090614AE0B4010D7B907C0130310A7B24BE
:106370007C0380047B207C03207938904C41E0B47E
:106380008431C003C004740212E4CE74509B5002E6
:1063900074FF0475F00AA4FA740C12E4E2EB2AFB11
:1063A000EC35F0FCD0F0D0E0FA9BE5F09C50048A8C
:1063B00003ACF0740E02E4EF2031012290614AE058
:1063C000B4020F90614DE075F014A40404FBACF02E
:1063D00080047B007C00741002E4EF741012E4E28D
:1063E000FD8B02741A12E4E2CB2ACB3DFC7412023C
:1063F000E4EF740212E4CE1475F00A30790375F0FC
:1064000000A4FBACF0741402E4EF740012E4CE14A8
:1064100075F014A4FBACF0741602E4EF740C12E4F3
:10642000E2FD8B02740E12E4E2C3EB9AFBEC9DFCDE
:10643000741802E4EF740012E4CEB41900501CFA90
:106440001A740112E4CEB4190040027418C39A758C
:10645000F014A4FBACF0741A02E4EF227B007C1869
:1064600090614AE0B4020B90614DE0203103FC8062
:1064700001FB741C02E4EF7E007F613031047E2456
:106480007F6122904C01E020E23790614AE0F97B85
:10649000503079107B84904C41E0B450077B50B968
:1064A00001027B84B90103EB03FB7C18B9020D9058
:1064B000614DE0FC303105C374189CFC741E02E48D
:1064C000EF904C41E0FB7C182079F17B5080ED2E61
:1064D000F582E43FF583E0FB222EF582E43FF5836D
:1064E000EBF0222EF582E43FF583E0A3FBE0FC22F3
:1064F0002EF582E43FF583EBF0A3ECF022E309B93B
:10650000020205A0F0A3DDF52275A0597900904C98
:1065100043E075F010A42410F582E5F03459F583BA
:106520007D1080D9904C43E075F010A42410F9E55B
:10653000F03459F5A09059007D1080C1904C42E094
:10654000F5F0904C41E0904D41303103904E41F0D8
:10655000A3E5F0F0904D3E303103904E3EE0A2793D
:1065600092E1F022904D41303103904E41E0F5F040
:10657000A3E0904C42F0904C41E5F0F0904D3E305D
:106580003103904E3EE0A2E19279F0229067F8E468
:10659000F090614AE0702690614EE0049067F8F058
:1065A000904C01E0F5F030E20C906120E0B401285D
:1065B000906101803990614EE060198028B4023604
:1065C00090614DE09067F870057402F08017B41880
:1065D000257401F0906120E0701C906101E0B41816
:1065E0001574018012906144E0700B906125E0B455
:1065F000180474028001E4601A90611820F206B455
:10660000E00390613CF5F0E0B420080582E0B403BB
:1066100002800375F000906784E0202F266024C07C
:10662000F0C0037B00B4020990614BE0B402027B2E
:106630000220540512A65D800312A5DBD003D0F022
:10664000906784E5F0F090614AE090614BF022128F
:10665000E50812E71CC2E0F0904C01E030E223C2F2
:1066600052906120E06003B4010B906100E0B41926
:10667000005002D25212E708D2E0A25292E1F00298
:10668000E52312E722C2E0F090614AE070089061D1
:106690004EE0600E8012B4021590614DE06009B4C6
:1066A000180CD250C251800AC250D2518004D2502C
:1066B000D251C252906120E07016906100E0B4198E
:1066C00000500D906118E070050582E06002D25222
:1066D000C253906144E07016906124E0B4190050F8
:1066E0000D90613CE070050582E06002D25312E734
:1066F00008A25092E0A25292E1F012E711A2519248
:1067000006A25392E1F002E523906120E00582F0B9
:106710008017906144E00582F02403800C90612191
:10672000E08006906145E0240375F010A4241FF575
:1067300082E5F03459F583E022906148EEF0A3EF52
:10674000F022906148E0A3FEE0FF2290E7D2E53B13
:10675000F0A3E53CF0A3E53DF0A3E53EF0A3E53F63
:10676000F0A3E540F0A3E52AF0A3EFF02290E7D2F2
:10677000E0A3F53BE0A3F53CE0A3F53DE0A3F53E47
:10678000E0A3F53FE0A3F540E0A3F52AE0FF2230C7
:10679000725312FD0790EC0130310390EE0175F059
:1067A000137917C00612092CD0067D048583A0A991
:1067B000827C00C2D112E7E512E82312E84212E817
:1067C0007AECF40412E813749CF30D90EC00303171
:1067D0000390EE00EDF0905FC0303103905FC1E0B8
:1067E00054F34404F02290E8B2E49360F8FAA3E48E
:1067F00093F8A3E493A3C083C082F583888230D149
:106800000012EA13F08004E012E813A3DAF0D08259
:10681000D08380D5FB12E819EBC4540FD2E6F32CD9
:10682000FC090D2290E8D1E49360BAFAA3E493F84E
:10683000A330D10612EA13F68004E612E81308DA50
:10684000F080E490E8E0E493609BFAA3303102A387
:10685000A3E493F8A3E493203102A3A3A3C083C0CD
:1068600082F583888230D10612EA13F08004E012A8
:10687000E813A3DAF0D082D08380CB75F00290E8E1
:10688000F0E493602DFAA3E493F8A3E493A3C08308
:10689000C082F583888230D10DEAF4FAE052021208
:1068A000EA134AF08005E05A12E813D082D083D56B
:1068B000F0CF22012B4C072D4C09444C0D504C01BC
:1068C000714C01D84C18134C01434C02005902037F
:1068D0005900012D012E012F01300133013802062C
:1068E000000E005045501115505A50017D51BD51B8
:1068F000003F2C4C60344C00904C93E0F5F090EC51
:106900001230310390EE0012712CEDF005F002967A
:106910002D206B9E904C93E07AD0B502951A1A7C8C
:106920000090EC0030310390EE00E02CFCA3DAFA8A
:106930008583A0A98212EA132C60012290EC7D309D
:10694000310390EE7DE020E30830770B12EF0080FA
:106950000620770312EF11904C43E0F53BE4A27957
:1069600092E0F53C12EBEE12F2A712EA1F12E7E5F5
:1069700012E82312E84212E87AE530781212FC0D90
:1069800012EC2412FC20307706E53B904C43F012C9
:10699000F2A712466312EC3874003031027401FC25
:1069A000FD12EA5312A47712A48612A5C712A500FD
:1069B00012A537E53C20790830E00B12862E8006C0
:1069C00020E00312862A12EA1FE92472F990E8CA2D
:1069D00012E7E812EBEE904C4212EA3090590012A6
:1069E00036FC905904E0F53B12EA30905903123618
:1069F000FC12EC05905905E0904C41F0FD1235D6A3
:106A000090FCB912460112133C1238C85333FE7B76
:106A10000102A5C3E309540FFBE309540FC44B2241
:106A200090EC0030310390EE008583A0A982D2D192
:106A300022E0FD904C43E004FB2275A05079A99020
:106A4000508A7A1E12F3B875A05379009052007ADA
:106A50000002F3B8ECA2E012EDCC12EC2412EC45EB
:106A6000EC6007904C01E020E20312EBF38C001283
:106A7000EC64782CE6F0080582B839F812413F75CD
:106A8000A04C792B904D2BBC0103904E2B7ACD124C
:106A9000F3B88D0012EC64782CE0F6058208B83962
:106AA000F8904C2B75A04D792BBD010575A04E7942
:106AB0002B7ACD12F3B8124128ED6007904C01E01B
:106AC00020E20312EC0A12EC5412FC20EDA2E09238
:106AD00031FB12A5A8D20912F9D402EC3812F2A7A0
:106AE000E4A23192E0FCB231A23192E0FD12EA530D
:106AF00012F2A7C322904F99E070F9E53920E2F431
:106B0000004C01E020E2ED20480C90688CE070061B
:106B100090688DE0600912F3BF400302EBBF229042
:106B20004BF4E0601120310520E008800320E103F0
:106B300002EBBF02C7F412F3BF403C904D2B203153
:106B400003904E2BE020E4781255865073A231B3A7
:106B500012EC8DE020E39D9068C22031039068C460
:106B6000E07009B23112556FB2315088904BEF741A
:106B70003CF0804C02EAF3904C2BE020E4F620033A
:106B80000C1255865007904BEF743CF022A231B3A3
:106B900012EC8DE020E3F5B23112556FB23150198D
:106BA00012F2EA40E790688C30310390688DE07013
:106BB00008904BEFE0600314F022904BD37420F068
:106BC00012F2EA407312EC24E4A23192E0FCB39298
:106BD000E0FD12EA5312C7F4904F9F303103904FFB
:106BE000A0E06005E4F01273F212F2A702EC381292
:106BF000FE2A4044904C43E0F812EC6E75A059799F
:106C0000EE7A1002F3B812FE2A402D12EC24904CBA
:106C100043E0F812EC6E8583A0A9829059007A10A7
:106C200012F3B88014904BE5E0B4020050087401F0
:106C3000F0E0B402FC2204F022904BE5E0B4020341
:106C4000E4F02214F022904C4DEEF0A3EFF0A3E517
:106C50003554F0F022904C4DE0FEA3E0FFA3E0534A
:106C6000350F423522904D00E86003904E0022908F
:106C7000EC81E82312712CE493F8A3E493F5838864
:106C80008222105920593059405950596059904F1B
:106C90008D5003904F8E2275A04D792B30310575A4
:106CA000A04E792B22905200500390530022A23123
:106CB00090508A50039050A922904D2B3031039070
:106CC0004E2B2290501530310390505A229050266E
:106CD00030310390506B22904AC5303103904B4ABB
:106CE000221253FEBD0A0302EDBD206666207563C5
:106CF000E53720E35EED20770CB411004001E4900D
:106D000031D1027141B40D4B904C2DE030E00312B3
:106D1000EF860246940278A5027996D25178010254
:106D20007ACBD2517801027BAA128184E53720E028
:106D30000930E1091280F3433702027FC31280C693
:106D400040F2A27F9251C27F7801127EE1A251925D
:106D50007FC251221237CBD269127D4FC2697B05A7
:106D600002A4D8024767206C030288A70288AE12EB
:106D70008184E53720E00930E1091280F3433702CE
:106D8000027FC31280C640F212ED9BA80718AD0621
:106D9000D269128B3CC2697B0502A4F9127A2612D1
:106DA0008C8DC39FF5F07A008531838532824383D1
:106DB000800AA3E054F665017003D5F0F422904CEC
:106DC0002FE030E719A23112EDCC021332904D3D85
:106DD0005003904E3DE0540C5330F34230227B057B
:106DE0007C08E53020E2027C0DAA0390EC013031F2
:106DF0000390EE01EC83F0A30CDBF9028F129B3FB2
:106E00000B30689B3F31306CC2D5904C43E0C0E002
:106E1000780110D5051238798003123802904C435E
:106E2000E0D000B50001221247671280F30213324E
:106E3000D2D580D6204135904C30E030E01512F9A3
:106E400038B4010A12F38A500512787E8024C250A9
:106E500002F8B47A0190EC0130310390EE017493A2
:106E6000F0128F1212F938B401BC8006BD0EB712B1
:106E700046E7BD0EB1024694204156904C30E030BA
:106E8000E005D25002F8B4904C31E030E50C12EE3F
:106E9000A67493F30912EEB4800912EEA612EEB4B2
:106EA0007493F30A028F1275A0EC790130310575E5
:106EB000A0EE790122904FAE303103904FB1E0FA4D
:106EC000A3E0F8A3E0F5838882A802E0F3A309D841
:106ED000FA22D0EE14ED17ED1AED21ED28ED53ED69
:106EE00062ED65ED6EEDBDED07EE2FEE33EE33EEA8
:106EF00077EECE7F307143904C2DE030E53CB8000A
:106F0000B8307736C27712EF1602EC05B8012B20A5
:106F1000772812EBEED27712A66512F00D12F9D493
:106F200012A47702A495307111E8B40300500BC489
:106F3000F8904C2DE05430B5000122307707C000A6
:106F400012EF00D000904C2DE054CF48F07802C0F2
:106F5000E012FC0DD0E030E51912EF1112C7A07558
:106F60003300C26EC26F12458C12EF0012EFF312A3
:106F7000EF7402133C12ECD67A85E4F0438380F080
:106F800053837FA3DAF52212EF7412F9D07B020249
:106F9000A59F904AC55003904B4A7A85E4F04383FD
:106FA00080F053837FA3DAF5021332904BD2E07066
:106FB00036D2D5904AC5302603904B4A20D503439C
:106FC0008380AC83AB82904A4020D5034383807A90
:106FD00085128D06E0128D05F0128D05DAF610D5BA
:106FE000D2904BD17401F02275A04C79DC904CE921
:106FF0007A0B800A75A04C79DA904CE77A0D12F37F
:107000007012722A904CF7E054014412F02212F2EE
:10701000A7904CE7E0CEF0A3E0CFF0A3E0C533F0BB
:10702000A3E054C0F8E52DF0532D3FE8422DA3A373
:1070300075A04C79447A0912F0B975A04C79D17ACF
:107040000212F0B9E0A2E0C0D0A27892E0D0D092D3
:1070500078A2E1C0D0A27F92E1D0D0927FA2E5C019
:10706000D0A27D92E5D0D0927DA2E6C0D0A26D9252
:10707000E6D0D0926DA2E4C2E4A830C854104853C0
:1070800030EF5003433010A2E2F8C083C082904C2E
:107090002DE0C0E092E1F0D0E0D082D083A2E1E820
:1070A00092E2F0904C5075A04C79DA7A0D12F0B95A
:1070B000E52F781312FC0D0283EEE3F8E0F3E8F01D
:1070C000A309DAF62220110C904F99E07006905F28
:1070D000DFE0600122905F32E0B44012905FD7E0C1
:1070E000F8905F34E0454730E008C820E70302F13C
:1070F00045C830E108C830E70302F145C8E8547FCD
:10710000900302F14A904F9DE0FDB4FF0122A3E0FD
:10711000CDFA904F9D74FFF0EA7006BD7F0C02F12E
:10712000F4BD0D0302F13702F1ABBDF20302F137FA
:10713000BD290280F802787AE87D0130E7027D02FD
:10714000905F34E04DF0C248D24922E830E720E5B4
:107150004730E008905F4D12273E500512F237800D
:107160000312F23EE4905F00F0905EC0F0801EE5F6
:107170004730E108905F5012273A500512F22580FF
:107180000312F233E4905E60F0905E80F07D0912AD
:107190000DA290CA527D3E12F19F12F21E02F0C45F
:1071A0007410F07430A3F0DDFC0212EC7A3F791118
:1071B000E8905E8030E703905EC0ED54606009B4F3
:1071C0007F028004E0B5020302787A04F0FB1271BA
:1071D0002CEDF0904A40E912712CEB12712CEDF07D
:1071E000EBB50202800C438380E06420F0A3E064EE
:1071F00020F00212EC7A3F7912E8905E8030E703CB
:10720000905EC0E0700302787AFB14F0904A40125E
:10721000712CE912712C7420F0EBB502C980D39067
:107220005FD7E004F0227941905F4D7420F0A3F025
:10723000A3E9F022794280F07942905F5080EC79A6
:107240004180F7905FD7E0F8547F60E77D09120D29
:10725000A290CA527D3E12F19FE820E705905E8021
:107260008003905EC07C00E060C9CCF0A3C083C006
:1072700082E0FD12F1ABD082D083A3DCF022907FBC
:10728000727401F012F2CA907F72E070F722907E61
:107290007EC001E0F9A3E069D00122907F7012F274
:1072A0009070F812F2B9C322202FF012A30170F8E7
:1072B00012F28D600512F2CA80F6907FF77401F029
:1072C000907FF7E060E112F2CA80F5124AB0C0F098
:1072D00012A711125975D0F002F3F612F2CA204A21
:1072E00006E53920E20122D3027310202FAD12F2FD
:1072F000DA12A30170F512F28D600512F2DA80F64F
:10730000907FF77401F0907FF7E0600512F2DA8069
:10731000F512F2DAC32290604930310390604AE4FA
:10732000F05337F712F34F904BE1303103904BE3BA
:10733000E4F022302F1A904F8CE020E00530260533
:10734000800E30260B907E7E12722A907F00E4F031
:10735000907EFE74FB303105907DFE74EF523A74DE
:1073600080F0A3F0907CCCE0203104C2E08002C227
:10737000E1F022531BDF431B40023BCF531BBF43B3
:107380001B2080F512F38A40E98016207729905956
:1073900000E0CEB50600CE4007905901E0B50600EA
:1073A00022207713905903E0CFB50700CF40079014
:1073B0005904E0B5070022C322E3F009A3DAFA2258
:1073C000C3203105202605D3222026FB2278003059
:1073D00031097803904C01E020E21B904C3FE0FB28
:1073E00075A0597C008C01C00012EC6ED0007A06AA
:1073F00012F3B808DBEF22906789E06024A3E0FD78
:1074000000629730E703906298E0FA1252C79067E3
:107410008A5008EBF0A3EDF0E4800274FE906789D7
:10742000F022070000000030001400390011400075
:107430000000002D001440000000002F0017400045
:1074400000000700000007000000400000004000AE
:10745000000080344C054000000040000000002F78
:1074600000160030001700300015400000004000FA
:107470000000802D4C100700000007000000002EC7
:107480000010002F001107000000802B4C17002D6A
:107490000016002F0015802E4C150700000000304C
:1074A000001300300016070000000030001080308C
:1074B0004C1007000000802F4C170700000080329E
:1074C0004C1080324C040700000007000000070049
:1074D00000000700000007000000802D4C0107009D
:1074E0000000070000000700000007000000070080
:1074F0000000070000000700000007000000070070
:10750000F70007000000070000000700000041002E
:107510000000070000000700000007000000002F27
:10752000001080334C1680334C1280334C13803360
:107530004C1180334C1707000000070000000700C3
:1075400000000700000007000000003000110700E5
:10755000000007000000070000000700000007000F
:10756000000007000000002F0012002F001307008A
:10757000000007000000002F0014070000000700B3
:107580000000802F4C15802E4C14070000000700CF
:10759000000007000000070000000700000012F5CF
:1075A000A512F5BE8036206B1230721075F0009077
:1075B0004C82E0B40103D2F022500122D26B22208F
:1075C0006B1920F016907D0E303103907D46753694
:1075D00008E4F0740712712CD536F622206B0FE503
:1075E000F0904C93F0904CC3E4F074088002740661
:1075F00002743D206BE5904C93E0F5F0BD3B3B20E1
:10760000132E30F62B30F428907D07E536F0904CA1
:10761000C3E0C0F075F00EA4D0F0907D0E303103C1
:10762000907D4612712C75A07D79007A0E12F3B808
:10763000904CC3E4F053F0008039BD2F0280092044
:10764000F79920F63802953030F404D2F780B9303B
:10765000F30CD2F4C2F2907D00E536F08015904C28
:10766000C3E0128CBA14B40400500E904CC3F0D294
:10767000F6D2F375360002962DD2F780F9E536B4CE
:107680000601221294D120F52920F209C4FA12F63B
:10769000A3EAF0800BFA12F6A3E04AF0D2F1053625
:1076A000B2F28015907D0130F403907D08E536023A
:1076B000712C30F102C2F5D2F780BB12F5C4780408
:1076C000907D0E303103907D4679317A047B15EB45
:1076D00083F0A30BDAF9E9F0A30909747EF07409C9
:1076E00012712CD8E622059B323412F6F012F7AF55
:1076F00022C2D590F01374B7F07C0512F74990F0D0
:10770000F77437F010D52320F61C12F74910D51A5C
:1077100012F8307401123B6A30920C12F822740194
:10772000123B6A2092042212F822431F4022BA0917
:107730001579F020D507741029F9B990012212F7B4
:10774000E712F76080ED798080F47AFF20D5040A93
:10775000BA0A012212F7C57420123B6A12F72D8073
:10776000EB12F81890F001E030E03890F010EC23C4
:10777000FCF07B2DEA540F2B83123B6A90F001E062
:1077800030E1205438701C90F000E06CB950028059
:107790000CB960028007B970028002C2E77004125F
:1077A000F81422D2D522A874542A150B060302011C
:1077B000904C0CE0F9FA12F81412F7E712F7C51220
:1077C000F81812F8222290F7DDEA540F93FB90F09C
:1077D00003E090F002E0EB447090F012F02201021E
:1077E000040506070A0C0E0F12F814E9C4540F9092
:1077F000F8009310E007C22090F012F022D220800F
:10780000704A7A5A4F4E4E7E5ECAFADACFCECEFE1C
:10781000DE7804800678008002780590F003E0545A
:10782000FA8008782090F003E0C2E54890F013F069
:1078300022780080F020776220680EE8705C90501B
:1078400000303103905045F022E534B40700400287
:107850007406905000303103905045F08028207716
:1078600018206816E86029B40600500D90F8999326
:10787000F8740112F88FA3E8F022E534B407004051
:1078800002740612F88FFAA375A04C798202F3B83D
:1078900090500730310390504CF0220C03040D132C
:1078A0002077F7E53030E3F212F938B4010512F32E
:1078B0008A40E7C2502041E212F8EA10500512282F
:1078C0002C80031228308030222077CE904C8212F8
:1078D000FB5212FBB640C312379012F8EA10500365
:1078E00002283902283922D25080DE1237903031F6
:1078F00004D20F8002D20B22D23412F938604E1417
:10790000D10D124694904C2DE030E0410246E71232
:107910008184E53720E03620E108127974500612A0
:10792000F9D00280F3905901E0B5060302F9D09036
:107930005903E0FF1246E780E9207E08E53020E5A4
:1079400005740222E53020E602E422740122207749
:107950002190590875F003800690590675F00212BF
:10796000FA21E0F8A3E0F583EF142850020583F52F
:107970008222C2D5D2D1D209C001C00212F983D06D
:1079800002D00122904AC6303103904B4BE583AAC6
:1079900082127E76127E7610D5E9F53110D103027F
:1079A000FA0102FA0D80DD2077FB90590675F0028E
:1079B00012FA21E0FAA3E010D576F53110D14FEE9E
:1079C00012712C74202582F58274013583F5838031
:1079D00032C204C26F53D0DD2077CA90590875F0C7
:1079E00003E0F8A3E0F5838882EE14A42582F582F3
:1079F000E5F03583F583E0FAA3E010D533F53110D7
:107A0000F00CA3E0F53554C0C2606002D260EF1400
:107A10002A50020531F532F58285318310091102B1
:107A2000A426E0F8A3E0F583850082EE1402B2A557
:107A30002253D0DD30770302F98390590875F003A3
:107A4000E0F8A3E0F5838882EE14A42582F582E5B0
:107A5000F03583F583A3A3E054C0C2606002D26016
:107A60002220411B1255F550161253E7905F32E069
:107A7000F8602A30320A12552F12214E2032E222AB
:107A8000BD140812552F12228480D6B84000400D34
:107A900012552FE54720E42920E54680C420261210
:107AA0001255FA50DABA400050D5124C3612552F02
:107AB00080AF12560850C8BA400050C3124D2780FC
:107AC000EC1255FA5008124C3612FAFA8093123121
:107AD0005320E24212FB0F7D3112FB227D0A020D80
:107AE0008E1256085008124D2712FB1D80DE1231EF
:107AF0005320E32212FB167D3280DE905F24E014D7
:107B000090B4FF12A3E014F030E70BE582B4250730
:107B10001231534404F0221231534408F022905F92
:107B20002680DBED905FE5F07D047430905FE1F03E
:107B3000A3DDFC222222128B2660FA904C41E00346
:107B4000F87484C398FA028C25222222222222224F
:107B5000904C83E0FDA3E0F8A3E0F9A3E0FA22C291
:107B600050127CAA502912F38A5003D25022E82ADC
:107B7000FA905903E014B500004001F8905904E070
:107B8000B502005001FA14B5000040DFEA98FA226D
:107B900012FBE1BA0001FAB8000108EAB5000040A2
:107BA0001512FBE1B502005001FAB500005001F8D2
:107BB000EAC39804FB182212FB8F40FA904C42E073
:107BC000FCB90001F9BD00010DE9B505004012EC5A
:107BD000B501005001F9B505005001FDE9C39D0450
:107BE000FC22904C41E02212FB4F753B8012FB8F30
:107BF00012FBBBE82B14F9ED14FA2C14FB02A5E3DD
:107C0000F2517D3031039051BDE04859F022C0E07F
:107C1000904D2B303103904E2BE812712CD0E0F0B8
:107C200022904C2BE0540790FC5B93532EE0452EA2
:107C3000F52E207326904CC2E4F020701ED27FE512
:107C40003030E31054F34404F530904D3D303103AF
:107C5000904E3DF0C00512EF00D005220717031328
:107C6000080100904C01E0A2E020E104303101B3B2
:107C700022904C01E05403905FC210E107F0A3B2E0
:107C8000E0F08003F0A3F0905FC212FC9B905FC213
:107C9000F0905FC312FC9B905FC3F022E0F8904C21
:107CA0000430E003904C08E0540FB405004009B4E0
:107CB0000A005004E8D2E122E82212FD46E0F9A3CE
:107CC000E0FA30D10DE9C4540FC9540FCA54F04A38
:107CD000C4FAE9F2E82410F8EAF2E824F1F810D145
:107CE00003D2D1A3DBD775A062785C796C7A10E3FC
:107CF00054F0C423FBE2540FCB2B75F00384C44B28
:107D0000310809DAEA02A670905191202E03904CB6
:107D1000137B18E4F0A3DBFC12FD46E2540FF9E8F4
:107D20002410F8E2FAE824F1F830D10BEA54F049D3
:107D3000C4F9EAC454F0FAE049F0A3E04AF010D1E3
:107D400003D2D1A3DBD522905191202E03904C1366
:107D500075A062785CD2D17B102212314DB4400DF7
:107D6000905F22E07007905F44E0B4300122E54765
:107D700030E02112315354C47018905F35E0701216
:107D800012FDB9400D742B7D001231C5905F241295
:107D9000FDB2E54730E1D612315354C870CF905F41
:107DA00035E070C912FDD540C4742B7D011231C578
:107DB000905F267A007B50022815905FC9E0FAA3F5
:107DC000E0F9905F24E02A400C54807007A3E0297A
:107DD0007002C322D322905FCFE0FAA3E0F9905F54
:107DE0002680E27B0012A5C3904C01E09000007B4E
:107DF0005A7990784830E20720312F7890800A3005
:107E0000F0079025207B5B7968E875F084A4FA057B
:107E1000F0E4F0438380F053837FA3DAF5D5F0F2EA
:107E20008B838982A3A3F0A3D8FA22C330310890B0
:107E30004C01E030E201D322306C2E904CD6EFF0B2
:107E4000128C8DC39FF5F0853183853282E060030B
:107E5000B42011438380E0700B53837FA3D5F0EDF2
:107E600074018001E4904CD7F02212FEA6500F203E
:107E70004133905FC2302603905FC3E0A2E12290BD
:107E80004C01E0A2E020E104302601B322905FC261
:107E9000302603905FC3E0904C0330E003904C0722
:107EA000E054077017D322904D2B302603904E2BB1
:107EB000C0E0E020E204D0E0D322D0E0C322904D25
:107EC0002E302603904E2EE0F57EA3E0F57F229023
:107ED0004D2B302703904E2BC0E0E05407B4060032
:107EE000D0E022740902743D206B1690EDFC303115
:107EF0000390EFFCE0B40300500804F012712CED85
:107F0000FF22D26B22B8010302E78EB802F602020A
:107F100008B80103020298B802EA02088FFFFFFFC7
:107F2000FFFFFFFFFFFFFFFFFFFFFFFFFFFFFFFF61
:107F3000FFFFFFFFFFFFFFFFFFFFFFFFFFFFFFFF51
:107F4000FFFFFFFFFFFFFFFFFFFFFFFFFFFFFFFF41
:107F5000FFFFFFFFFFFFFFFFFFFFFFFFFFFFFFFF31
:107F6000FFFFFFFFFFFFFFFFFFFFFFFFFFFFFFFF21
:107F7000FFFFFFFFFFFFFFFFFFFFFFFFFFFFFFFF11
:107F8000FFFFFFFFFFFFFFFFFFFFFFFFFFFFFFFF01
:107F9000FFFFFFFFFFFFFFFFFFFFFFFFFFFFFFFFF1
:107FA000FFFFFFFFFFFFFFFFFFFFFFFFFFFFFFFFE1
:107FB000FFFFFFFFFFFFFFFFFFFFFFFFFFFFFFFFD1
:107FC000FFFFFFFFFFFFFFFFFFFFFFFFFFFFFFFFC1
:107FD000FFFFFFFFFFFFFFFFFFFFFFFFFFFFFFFFB1
:107FE000FFFFFFFFFFFFFFFFFFFFFFFFFFFFFFFFA1
:107FF000FFFFFFFFFFFFFFFFFFFFFFFFFFFFFF335D
:00000001FF
